:100000000C9484170C94AC170C94AC170C94AC178C
:100010000C94AC170C94AC170C94AC170C9485335F
:100020000C94AC170C94AC170C94AC170C94AC1744
:100030000C94AC170C94AC170C94AC170C94AC1734
:100040000C94152F0C94AC170C94EE300C94AC1748
:100050000C94AC170C94AC170C94AC170C94AC1714
:100060000C94AC170C94AC17071B091B091B091B3C
:10007000091B091B091B091B091B091B091B091B60
:10008000F51A091BB91AD71AAB1A2D1A3B1A491AB5
:10009000571A651A731A811A8F1A9D1A091B091BA0
:1000A000091BC91A091BE51A091B091B091B091B96
:1000B000091B091B091B091B091B091B091B091B20
:1000C000091B091B091B091B091B091B091B091B10
:1000D000091B091B091B091B091B091B091B091B00
:1000E000091B091B091B091B091B21192919351992
:1000F00041194B1951195D19671973197B19871922
:1001000091199D19A519AD19B719C319CF19D91985
:10011000E319E919F319FF19091A151A211A6F6B56
:100120003B0077783B0072783B0074783B00676453
:100130003B00646C3B0069733B006F703B00796C63
:100140003B0064653B0061633B0065723B00657387
:100150003B0037333B0063713B0068693B006F65D0
:100160003B00676E3B006F763B00776B3B00736F25
:100170003B0035353B0061743B0064783B006662B0
:100180003B006E6F3B006D793B0076793B00746FEE
:100190003B006F663B0065753B00766C3B00697405
:1001A0003B006D653B0063773B006A613B006F621B
:1001B0003B0064613B00696E3B006F6E3B00626B0D
:1001C0003B00646F3B0061673B00676F3B006174FD
:1001D0003B006B6D3B0073703B0062793B006862D3
:1001E0003B0070613B0064783B0075733B00646CBE
:1001F0003B0067743B00666D3B00616D3B00676EC2
:100200003B0067703B0068663B006C773B006E729A
:100210003B006E773B006F6D3B0072663B00736E78
:100220003B00766C3B00776C3B00796C3B003535CE
:100230003B0061733B001E01220126012A012E01B1
:10024000320136013A013E01420146014A014E01A6
:10025000520156015A015E01620166016A016E0196
:10026000720176017A017E01820186018A018E0186
:10027000920196019A019E01A201A601AA01AE0176
:10028000B201B601BA01BE01C201C601CA01CE0166
:10029000D201D601DA01DE01E201E601EA01EE0156
:1002A000F201F601FA01FE01020206020A020E0242
:1002B000120216021A021E02220226022A022E022E
:1002C0003202746E783B007372693B007173623B5B
:1002D000006162743B007269673B007769723B00A2
:1002E0006D69743B006469643B00756E733B007319
:1002F00068653B00636C723B00616E743B00747216
:10030000783B007073653B00746B733B006E696CE7
:100310003B006D69723B006469723B0078796C3B0D
:100320000074776F3B0071736F3B006665723B0032
:100330006861743B007761723B006872643B006CDB
:1003400074723B0069686D3B0077686F3B006375B2
:100350006C3B007761733B007075743B006275679E
:100360003B006572653B006561723B006F68723BE4
:1003700000626F783B006269673B00616E643B001E
:10038000756E643B006C6F743B0064656D3B00717F
:10039000736C3B0077726B3B0065696E3B00746861
:1003A000653B0071736F3B007369653B0071727050
:1003B0003B0071726F3B0071736B3B006F76763B55
:1003C000007377723B007275663B006C6F733B0085
:1003D000676E643B006169723B0064776E3B006648
:1003E0006F673B006E75723B00626F793B00736113
:1003F000653B0068616D3B006972633B00766F6E20
:100400003B006C6F773B006C65743B007566623B2C
:1004100000746F6F3B006263693B006B65793B0062
:100420007373623B00706B743B00746D773B0064C8
:1004300069653B006461733B006D6E693B007172DE
:100440007A3B007273743B006672713B0075736592
:100450003B0077706D3B0062706D3B006F6E653BDB
:10046000006269743B0073776C3B007270743B00F0
:100470006275673B006F75743B007768793B00716C
:10048000736C3B007668663B0076666F3B0071726A
:100490006D3B007476693B00766C6E3B006C62725B
:1004A0003B006D696E3B006469723B0063666D3BA7
:1004B0000061676E3B0071726E3B007172673B00BA
:1004C00066756E3B0073756E3B00616D703B00712D
:1004D000726C3B006C65643B00616C733B00646153
:1004E000733B006465723B00C202C702CC02D102BA
:1004F000D602DB02E002E502EA02EF02F402F902B0
:10050000FE02030308030D03120317031C03210358
:1005100026032B03300335033A033F034403490307
:100520004E03530358035D03620367036C037103B7
:1005300076037B03800385038A038F039403990367
:100540009E03A303A803AD03B203B703BC03C10317
:10055000C603CB03D003D503DA03DF03E403E903C7
:10056000EE03F303F803FD03020407040C04110473
:1005700016041B04200425042A042F04340439041F
:100580003E04430448044D04520457045C046104CF
:1005900066046B04700475047A047F04840489047F
:1005A0008E04930498049D04A204A704AC04B1042F
:1005B000B604BB04C004C504CA04CF04D404D904DF
:1005C000DE04E30468616E643B00776972653B009A
:1005D000686175733B00746861743B007361736597
:1005E0003B006D616E6E3B00736E6F773B00646124
:1005F00063683B00726F6F663B006371646C3B0025
:100600006D6173743B006C6573653B006D6F737453
:100610003B00776572653B0064616E6E3B0066650A
:10062000696E3B0074656D703B007365656E3B00E1
:10063000726376723B00726376643B0073616D6532
:100640003B007761726D3B00636F6F6C3B00786DB0
:1006500074723B00626F79733B007468656E3B0097
:100660006D6164653B00627563683B007863757318
:100670003B007768656E3B0077726B643B00676593
:1006800062653B00737563683B00666F6E653B0097
:10069000686162653B007265696E3B00676568650D
:1006A0003B007A61686C3B006562656E3B00677277
:1006B00061643B006265656E3B0066616C6C3B008B
:1006C000686F6D653B00636F6E643B0064616E6EC6
:1006D0003B00746869733B00746861743B00647824
:1006E00063633B00657264653B0063616C6C3B0057
:1006F00064696E673B006D6163683B006D6F726596
:100700003B00727474793B00616C736F3B006D69E0
:1007100073743B00637264733B00646F72743B00DC
:1007200064616E6E3B00717565723B006D6F76653E
:100730003B006F7665723B00616265723B006461ED
:1007400073683B00646F63683B00646172633B00E5
:100750006C696B653B00727072743B00696872650E
:100760003B006465696E3B00686F63683B00736BB8
:1007700065643B00736967733B006E65696E3B009F
:100780006D6568723B00667573733B0066756E6BD2
:100790003B0064656E6B3B0064616E6B3B006B728B
:1007A000616E3B006E65696E3B006265616D3B008A
:1007B00069636F6D3B00736173653B007874616CB6
:1007C0003B00777474733B00696E666F3B00626335
:1007D0006E753B00617764683B00696E70743B0026
:1007E0006270736B3B00686F63683B007469656699
:1007F0003B00616265723B006E6F63683B0079612C
:1008000072643B007365656E3B0062616E643B0021
:10081000626572673B006D6565723B007369656771
:100820003B006172726C3B006D6965663B00616400
:1008300065723B007765696E3B0073656B743B00C6
:100840007A61756E3B006B61756D3B007261756D11
:100850003B006A756D703B00C405CA05D005D6051E
:10086000DC05E205E805EE05F405FA0500060606D6
:100870000C06120618061E0624062A063006360640
:100880003C06420648064E0654065A0660066606B0
:100890006C06720678067E0684068A069006960620
:1008A0009C06A206A806AE06B406BA06C006C60690
:1008B000CC06D206D806DE06E406EA06F006F60600
:1008C000FC06020708070E0714071A072007260769
:1008D0002C07320738073E0744074A0750075607D8
:1008E0005C07620768076E0774077A078007860748
:1008F0008C07920798079E07A407AA07B007B607B8
:10090000BC07C207C807CE07D407DA07E007E60727
:10091000EC07F207F807FE0704080A081008160893
:100920001C08220828082E0834083A0840084608FF
:100930004C085208676C617562653B006E696368BC
:10094000743B00696D6D65723B0077696564657223
:100950003B0066756E6B656E3B00616E74656E6E16
:10096000653B006469706F6C3B006C616E6764721C
:100970006168743B0068696D6D656C3B00617574FE
:100980006F3B0066616872656E3B007472656666F7
:10099000656E3B006B6162656C3B0066696E646509
:1009A0006E3B006B617566656E3B00696E746572C7
:1009B0006E65743B0072656C6169733B006C616EBF
:1009C00067796167693B0064726568656E3B0072B8
:1009D0006F746F723B0067726F756E64706C616EDE
:1009E000653B006B61656C7465723B007765747480
:1009F00065723B00736F6E6E653B00726567656E76
:100A00003B006765736568656E3B006C616E67658A
:100A10003B0074657565723B007072756566756E36
:100A2000673B0073746174696F6E3B0073656E643D
:100A300065723B0079616573753B00656C65637237
:100A40006166743B006B656E776F6F643B00676532
:100A500061726265697465743B00656E6473747578
:100A600066653B006C65696465723B007369636829
:100A700065723B00676562656E3B006D6F7267650E
:100A80006E3B0073757065723B006665726E7365D0
:100A900068656E3B006D6F6E69746F723B00636FCB
:100AA0006D70757465723B00776F7274653B006C96
:100AB00065697374756E673B00626564696E67751E
:100AC0006E673B007363686C656368743B006265C6
:100AD000737365723B00637561676E3B0078637585
:100AE000733B00636F6E64783B00696E666F726D76
:100AF0006174696F6E3B006E756D6D65723B006A67
:100B000065747A743B0074617374653B0074656C42
:100B100065666F6E69653B0074656C6567726166DA
:100B200069653B0073706165743B0066727565684A
:100B30003B007370756C653B006B6F6E64656E7324
:100B400061746F723B0073706572726B726569736A
:100B50003B00666C696567656E3B006C697A656E23
:100B60007A696572743B0070726F626C656D3B00F0
:100B70007472696E6B656E3B00657373656E3B00E6
:100B8000656C6275673B0061776172643B0062650A
:100B900064696E67756E673B00686F6262793B00DF
:100BA000616D617465757266756E6B3B007361741F
:100BB000656C6C69743B006675737362616C6C3B49
:100BC00000747261756D3B006578706572696D6562
:100BD0006E743B00646575746C6963683B00736395
:100BE000687765723B006C65696368743B00756E7D
:100BF0007465723B007374756E64656E3B006D695D
:100C00006E7574656E3B006B6F6D6D656E3B006B52
:100C10006F7066686F657265723B006C61757473A6
:100C2000707265636865723B00696E666F726D69AC
:100C30006572656E3B00647275636B656E3B006D3B
:100C40006F72736574617374653B00636F6E746576
:100C500073743B00686F6262793B00766F726D69F6
:100C600074746167733B006C65697365723B006CFB
:100C700061757465723B00726164696F3B006475F5
:100C80007263683B00676567656E3B006D65746500
:100C9000723B006E6562656C3B00657572656E3B0C
:100CA0000077656E69673B007669656C653B00752A
:100CB0006872656E3B0073746966743B006573739C
:100CC000656E3B00736F6761723B00686562656CBF
:100CD0003B0074617374653B006B657965723B0022
:100CE0006861656E64653B0073656E6465723B00A8
:100CF0006C616D70656E3B0066696C7465723B007B
:100D00007469656665723B00686F656865723B0073
:100D10007765697465723B00736F7267656E3B003F
:100D200064756D6D65723B006172626569743B004C
:100D30007A696568656E3B00736F6E6E69673B002C
:100D4000686F6572656E3B00776F6C6B69673B001F
:100D5000676C656963683B006D75737465723B0011
:100D600066756E6B65723B0068656C6665723B000C
:100D70006272696566653B00626567696E6E3B001D
:100D8000616C6C65696E3B0066657269656E3B00FF
:100D90006C616E6765733B0066696E6465743B00E9
:100DA000676C617562653B006469706C6F6D3B00D8
:100DB000616E7465696C3B006D6F7273656E3B00AC
:100DC0007363686C61663B006B72696567653B00C5
:100DD0006B6F6D6D656E3B00667265756E643B0092
:100DE000686F657265723B006B617374656E3B0082
:100DF00073696562656E3B006272696E67743B0081
:100E00007363686164653B006B6F7374656E3B0070
:100E10006B61727465693B007361756265723B005A
:100E200066696E6765723B00616273696368743BF3
:100E300000747261656765723B0073746F657265FB
:100E40006E3B0067726F657373653B006C6F676222
:100E50007563683B007665726D65726B3B0068690F
:100E60006E776569733B00617262656974653B000A
:100E700066696E646573743B006E6F74697A656E43
:100E80003B0067656C6573656E3B006E6F63686DF4
:100E9000616C3B00766F726C6167653B006C616EE4
:100EA0006773616D3B007363686E656C6C3B007AC1
:100EB00065696368656E3B00676C65696368653B7F
:100EC000006461676567656E3B006672756568659D
:100ED000723B0064617565726E643B0067657261A8
:100EE0006574653B006765686F6572743B0062728C
:100EF00061756368653B006765737465726E3B007E
:100F00007A756B756E66743B006D6574686F6465A9
:100F10003B00617274696B656C3B0067656D616372
:100F200068743B006B6C696E67656C3B0077696346
:100F3000687469673B00736368776163683B00624C
:100F400072696E67656E3B007775657264656E3BAE
:100F5000006265736F7267653B006B6174616C6FF3
:100F6000673B0064756E6B6C65723B006C6165730A
:100F70007469673B007363686E6974743B007370D7
:100F800072616368653B00676564616E6B653B0019
:100F900061757373696368743B0073696E6E766F15
:100FA0006C6C3B0074617374617475723B006E61AC
:100FB00063687465696C3B00646168696E7465722E
:100FC0003B007665726B617566653B0067657769A6
:100FD0006E6E65723B0065726C65646967743B0098
:100FE0006D616E63686D616C3B0062616E64706C14
:100FF000616E3B007363687765737465723B00765E
:1010000065726C696572656E3B007363686E656CD2
:101010006C65723B0061626B7565727A656E3B0050
:10102000616D6174657572656E3B006E6F74697A8F
:10103000627563683B00766F726D65726B656E3BBF
:1010400000626C656973746966743B0067656E6104
:1010500075657265733B006772756E647361747A4F
:101060003B006265686F657264656E3B0067656E24
:101070006175657265733B006D6974686F65726553
:101080006E3B00616C6C67656D65696E3B006E6FF1
:101090007477656E6469673B006E6163687269634B
:1010A00068743B006765627261756368743B006BCE
:1010B00075727A77656C6C653B0062657275666CFB
:1010C0006963683B0077756E6465726261723B00AC
:1010D00064616368626F64656E3B0065696E736529
:1010E000697469673B00766F727A65697469673BFA
:1010F000006765726164656175733B007665726255
:1011000072617563683B00627563687374616265E0
:101110003B006D6568726D616C69673B0062657765
:10112000756E646572743B006861657566696765B4
:10113000723B006C616E646B617274653B00766536
:1011400072736F7267656E3B007765726B73746163
:1011500074743B006265697472616567653B006D1C
:10116000657373706C61747A3B0065696E7370723D
:101170007563683B00656973656E6261686E3B000C
:10118000776F6572746C6963683B006E6163686653
:10119000726167653B0061757373756368656E3B6B
:1011A0000062656D65726B6261723B00756E6265AF
:1011B0006B616E6E743B006E6F6572646C69636820
:1011C0003B00666F65726D6C6963683B00617066B9
:1011D000656C73696E653B00726F73656E62656501
:1011E000743B006D6F65676C696368653B00766F83
:1011F00072736963687469673B0073746F657265C5
:101200006E6465733B006E61656368746C696368E6
:101210003B00766F726D6974746167733B0067722F
:1012200075656E646C6963683B006E6163687465C4
:10123000696C69673B00756E676573746F6572747E
:101240003B0077756E646572766F6C6C3B006672FE
:10125000616E6B72656963683B0065696E73696393
:10126000687469673B007469656673696E6E696767
:101270003B0067726F737361727469673B007669D4
:10128000656C7365697469673B007472616E73693C
:1012900073746F723B006C6F65746B6F6C62656E1C
:1012A0003B006D6573736765726165743B007765BC
:1012B00074746265776572623B00676567656E731B
:1012C000656974653B0073757065726D61726B74EE
:1012D0003B0073746F6572756E67656E3B006C657D
:1012E000697374756E67656E3B00676573756E64D0
:1012F000686569743B00756E7465726B756E6674B3
:101300003B0066756E6B667265756E643B00697353
:101310006F6C61746F72656E3B00766572616272AC
:10132000656465743B00696E666F726D61746976A1
:101330003B00756562657273696368743B00766F24
:1013400072736368726966743B00676C7565636B82
:101350006C6963683B00667265756E646C6963688E
:101360003B006D6974676C69656465723B0061750B
:10137000666D65726B73616D3B0072756E64737040
:10138000727563683B0061626B7565727A756E6732
:101390003B00747265666670756E6B743B007769AE
:1013A0006465727370727563683B006461656D702B
:1013B00066756E673B006162656E6468696D6D6538
:1013C0006C3B00776F6C6B656E6C6F733B00756E7A
:1013D000667265756E646C6963683B007465696C00
:1013E0006E65686D65723B00666C6F686D61726BEF
:1013F000743B0072756E6473747261686C65723BE5
:10140000006665726E737465756572756E673B0014
:1014100061627370616E6E656E3B007565626572C8
:1014200074726167656E3B00646973706C61793BCF
:1014300000736F6E6E656E666C65636B656E3B0008
:101440006D6178696D616C3B00756E676C6175628A
:101450006C6963683B00706C6174696E653B006425
:101460007265686B6F6E64656E7361746F723B005A
:10147000766572626573736572756E673B0062654F
:10148000736368776572656E3B006E616368626165
:10149000727363686166743B00616C7465726E613F
:1014A000746976653B006F737A696C6C61746F72F6
:1014B0003B006261756D61726B743B0062617573B4
:1014C00061747A3B0065696E7374656C6C756E67E8
:1014D0003B00706172616D657465723B00686F639B
:1014E000687061737366696C7465723B00656D69E1
:1014F00074746572736368616C74756E673B0066C3
:10150000656C64656666656B747472616E7369732D
:10151000746F723B00726F746F727374657565726D
:10152000756E673B00736368616C746E65747A7482
:1015300065696C3B00727568657374726F6D3B0012
:101540006C657563687464696F64653B006B617496
:10155000686F64653B006C696368747175656C6C79
:10156000653B007369676E616C3B00736368616C17
:1015700074706C616E3B00706C6174696E656E6C4A
:1015800061796F75743B007A656974756E673B00AD
:10159000717561647261743B00706172616C6C653D
:1015A0006C3B0073657269656C6C3B00756D7363B1
:1015B00068616C7465723B0061757373696368740C
:1015C0003B007669656C6C65696368743B007365A4
:1015D0006C74656E3B0073746164743B0061757478
:1015E0006F6261686E3B007061726B706C61747ADF
:1015F0003B006469676974616C3B006B616D657287
:10160000613B007472616E736365697665723B005D
:101610007261737465723B00616C61726D3B006E48
:101620006F7466616C6C3B00706F6C697A65693BC6
:1016300000756D726563686E656E3B007A657273E6
:10164000746F6572656E3B0062616B656E3B007521
:101650006D7365747A65723B00617573627265695A
:1016600074756E673B006E6577636F6D65723B00E6
:1016700076657273746568656E3B00656D70666152
:101680006E67656E3B0073656E64656E3B007363E9
:10169000686C6166656E3B006E616368743B0061F7
:1016A0007566676577616368743B00776561746828
:1016B00065723B00736F6C61723B00666F726563AD
:1016C0006173743B00736F6C646572696E673B0095
:1016D0006D6F6E69746F72696E673B00696E7472CC
:1016E000756465723B007265706561743B00706F74
:1016F00072746162656C3B0064656E6B6261723B23
:10170000006865726273743B0077696E7465723B42
:1017100000736F6D6D65723B0066727565686C690C
:101720006E673B007363686E65653B006175736649
:101730006C75673B0062616E646272656974653BDB
:1017400000746165676C6963683B007374756465F8
:101750006E74656E3B0073636875656C65723B0003
:101760006C65687265723B006261757374656C6C60
:10177000653B006C6562656E3B0062617573746504
:10178000696E653B00756E76657273636861656D41
:10179000743B00726563686E656E3B006D697473BF
:1017A000636872656962656E3B007A75686F657221
:1017B00065723B006661636867657363686165664F
:1017C000743B0073746174697374696B3B00776573
:1017D00074746572626572696368743B00726567F0
:1017E00069737472696572656E3B007363616E6ED6
:1017F00065723B006E65757765727469673B006260
:101800006C69747A3B0077696E647261643B007541
:10181000726C617562736F72743B006B6F6D706197
:101820006B743B006665726E67657374657565728F
:10183000743B00616C6B6F686F6C3B00766F72730A
:10184000747566653B0034093C0943094A0952092D
:101850005A0963096A0975097D0983098B09940985
:101860009B09A309AB09B509BD09C709CF09D60969
:10187000E309EC09F409FB09020A0B0A120A190A26
:10188000230A2C0A340A3B0A450A4E0A5A0A640AF9
:101890006C0A740A7B0A830A8A0A950A9E0AA80AB5
:1018A000AF0AB90AC40ACE0AD60ADD0AE30AEA0A6E
:1018B000F70AFF0A060B0D0B180B240B2B0B320B30
:1018C000390B460B520B5B0B670B700B790B800BC4
:1018D000870B8E0B990BA00BAD0BB70BC10BC80B75
:1018E000D40BDE0BE60BEE0BF50BFE0B070C0F0C0F
:1018F0001B0C290C360C3F0C4B0C540C5B0C670C6E
:101900006F0C770C7E0C850C8C0C930C9A0CA10C34
:10191000A80CAF0CB60CBD0CC40CCB0CD20CD90C63
:10192000E00CE80CF00CF80C000D080D100D180D73
:10193000200D280D300D380D400D480D500D580D5F
:10194000600D680D700D780D800D880D900D980D4F
:10195000A00DA80DB00DB80DC00DC80DD00DD80D3F
:10196000E00DE80DF00DF80D000E080E100E180E2B
:10197000200E280E310E3A0E430E4C0E550E5E0E02
:10198000670E700E790E820E8B0E940E9D0EA60EB3
:10199000AF0EB80EC10ECA0ED30EDC0EE50EEE0E63
:1019A000F70E000F090F120F1B0F240F2D0F360F0C
:1019B0003F0F480F510F5A0F630F6C0F750F7E0FBB
:1019C000870F900F9A0FA40FAE0FB80FC20FCC0F56
:1019D000D60FE00FEA0FF40FFF0F0A1015102010BA
:1019E0002B10361041104C10571062106D107810EB
:1019F00083108E109910A410AF10BA10C510D0101B
:101A0000DB10E610F110FC10071112111D11281146
:101A100033113E11491154115F116A117511801172
:101A20008B119611A111AC11B711C211CD11D811A2
:101A3000E311EE11FA11061212121E122A123612B8
:101A400042124E125A12661272127E128A129612A6
:101A5000A212AE12BA12C612D212DE12EA12F61296
:101A600002130E131A13261332133E134A1356137E
:101A700062136E137A13861392139E13AB13B6136D
:101A8000C313CE13DC13E813F313011410141B1447
:101A9000281431144014491456145F1470147E1421
:101AA0008A149914A614B214BC14C514D214DD14EB
:101AB000ED14FF1415152515351540154D15561542
:101AC00063156B157715871590159915A315AC152A
:101AD000B815C215CE15D615DD15E715F215FB158F
:101AE0000316101618161F16281631163C1648161F
:101AF0004F165916661670167B1686168E16981691
:101B00009F161E12B416BB16C516D016DC16E616A6
:101B1000EE16F816011709171117191724172C17A5
:101B2000351741174B1756176017681773177A1731
:101B3000851793179C17AA17B417C317CE17DD176D
:101B4000EB17F417FF1706180F181B182418331873
:101B50003C18646C386B666F20646520646C316B74
:101B60006270203D20746E782066657220727072FB
:101B700074203539392066726F6D20636F6C6F6722
:101B80006E65203D20757220727374206973203554
:101B900037392035376E203D2071746820697320F5
:101BA0006E722061616368656E2061616368656E55
:101BB000203D206E616D65206973206672616E6BD9
:101BC000206672616E6B203D20687065206F6B3FF0
:101BD00020646C386B666F20646520646C316B62C6
:101BE0007020707365206B3B0077387973642064D4
:101BF0006520646C3274756E203D20616C6C2072BF
:101C000069676874206465617220627279616E2010
:101C10003D2071736C207669612062757265617513
:101C2000206F6B203D20746E7820666572206E698F
:101C300063652071736F20616E642061206E69633B
:101C400065207765656B656E64203D206870652052
:101C5000637561676E20736F6F6E203D20773879F2
:101C6000736420646520646C3274756E206E772016
:101C7000717274206520653B00646C366B626C2069
:101C800064652069356F7066203D206578637573E3
:101C9000206472206F6D2062656E203D2068722086
:101CA0006E696C20696E666F20616274206D7920A8
:101CB0006F75747074203D206D7920707772206D7F
:101CC0007472206E696C206F6B203D2070612074EF
:101CD000627320327836313436203D20696E70745C
:101CE00020616274203136302077747473203D2077
:101CF000646C366B626C2064652069356F70662099
:101D0000707365206B3B00646A316B6B6F20646598
:101D1000206561396D63203D20616C6C206F6B2004
:101D2000647220616C62657274203D20707365205E
:101D3000717270203D207572207369676E2076790C
:101D4000206764203D2072737420356E6E20356EDE
:101D50006E203D206D79207478206F75747074202A
:101D60006E7720322077747473203D20687720636B
:101D700070693F203D20646A316B6B6F2064652081
:101D80006561396D6320707365206B3B00646C3452
:101D90006661206465206862396C71203D206F6B3C
:101DA000206D79207369677320727374203436391B
:101DB00020736F2061676E206D6E6920746E7820CD
:101DC00066657220696E666F203D206D7920616EB8
:101DD0007420666572203430206D74727320322056
:101DE000656C207961676920736F20737572652057
:101DF000776C2063706920796F7520746D77206F20
:101E00006E2037303032206B687A203D20646C348D
:101E10006661206465206862396C7120707365208A
:101E20006B3B00646B396172206465206467386BBA
:101E30006372203D20746E78206665722063616C49
:101E40006C20647220667264203D20757220736974
:101E5000676E20727374203337386B203337386BDA
:101E60003D20717468206B617373656C206573200D
:101E70006E616D652077696C6C69203D20726967C1
:101E800020747276637220686F6D656D6164652081
:101E900066657220637720657320737362203D202E
:101EA00070777220616274203520777474732061BA
:101EB0006E74206469706F6C65203D2068772063C4
:101EC00070693F203D20646B396172206465206435
:101ED00067386B637220707365206B3B00646637F4
:101EE0006F6C78206465207061336572203D2076C8
:101EF0007920737269206472206F6D206B6C61753C
:101F000073203D206E696C206370692075722073A8
:101F1000696773203D2061676320696E206D7920B9
:101F20007472637672206E696C206F6B203D207036
:101F300073652035206D696E203D20776C206361CC
:101F40006C6C20752061676E20736E203D20616788
:101F50006E206578637573203D206466376F6C78FA
:101F60002064652070613365723B00646C3976676C
:101F700020646520646A33776173203D206775743F
:101F8000656E206162656E64206C696562657220B1
:101F9000746F6E69203D207363686F656E2064699D
:101FA0006368207A7520686F6572656E203D2064D5
:101FB00065696E2072737420697374203539392015
:101FC000356E6E203D2069636820686F6666652CFB
:101FD00020647520686174746573742065696E652A
:101FE0006E20677574656E207461673F203D2064C4
:101FF0006C39766720646520646A3377617320707A
:102000007365206B3B00646B3478792064652064D1
:102010006C376B7A6F203D206E65696E2C206D6980
:10202000636861656C206963682068616265206B24
:1020300065696E65206E65756520616E74656E6E8E
:1020400065203D20616E7420666233332066623302
:1020500033203D20667565722032306D20726569CF
:10206000636874206D69722064617320766F6C6C94
:102070006B6F6D6D656E206869203D2077616E6EB7
:10208000206B6F6D6D742064656E6E206465696E83
:10209000206E65756572206D6173743F203D20640C
:1020A0006B34787920646520646C376B7A6F2070AC
:1020B0007365206B3B007731617720646520646C29
:1020C000397A6D203D2073746E2068722037357424
:1020D0002077747473206F75747075742065732025
:1020E000616E74203520656C2079616769206162BA
:1020F00074203138206D7472207570203D207778FF
:1021000020756662207769642074656D70203330B5
:102110002063203D20707365207173792032206B1D
:10212000687A2064776E203D2068722071726D207D
:1021300066726D20727474792073746E203D207005
:102140007365206B3B006466346B782064652064A3
:102150006A316A77203D20676D206C627220756C51
:102160006C6920657320766C6E20646B20666572E6
:1021700020696E666F2061627420636F6E74657390
:1021800074203D20636F6E647320756662203D206D
:1021900070736520717271203D206D7920727820F6
:1021A000686F6D656D6164652077696420323320E6
:1021B000746273203D20777820666220323120637C
:1021C000203D20687065206177646820746D7720F9
:1021D0003D3D3B00646D39656520646520646B3866
:1021E0007A66203D206861626520686965722073A7
:1021F0007461726B65732071726D206475726368AF
:102200002065696E652073746174696F6E206175F5
:102210007320796F203D20696872206E616D6520A2
:10222000756E64206968722071746820776172200D
:102230006E69636874206175667A756E65686D6530
:102240006E203D20626974746520676568656E2044
:10225000736965207A756D2073656E64656E2035CF
:10226000206B687A20686F65686572203D206D6517
:10227000696E206E616D6520697374206B61726C8C
:102280006865696E7A20756E64206D65696E20716F
:102290007468206973742077616C6473617373650B
:1022A0006E206E72206F6B206772656E7A65203DBE
:1022B0003B007761327177206465206F6E35666B05
:1022C000203D206765206472206F6D20626F622060
:1022D0006573206D6E6920746E7820666572207556
:1022E00066622072707274203D2075722073696777
:1022F00073206872206E772072737420343739200F
:1023000034376E203D206D792073746E20747263B3
:1023100076722077696420313030207720696E70C2
:102320007420657320616E74206770203D20707387
:1023300065206B3B006B31777320646520646C32E1
:10234000777973203D206F6B2077696420696E6612
:102350006F20616274207572207269672064722038
:102360006F6D206A696D203D20687220726376640B
:1023700020616C6C206662203D2068772061627469
:1023800020736B65642066657220746D77206F6EB4
:102390002031306D203F203D2071727620696E2003
:1023A00073737476203D2071726B3F203D206B313A
:1023B000777320646520646C32777973207073655D
:1023C000206B3B006B613161626320646520707932
:1023D000306D6167203D20756662206472206672F0
:1023E00064203D207073652075722071736C2077B6
:1023F00069642073616520657320322069726320EF
:102400003D20776C2071736C20766961206469725D
:1024100065637420657320737572652063666D2033
:1024200073776C207270727473203D3D3B0066338D
:10243000747220646520646A39707771203D20755C
:102440007220727072742072737420353939203D95
:102450002073756D20717362203D20707772206843
:102460007220373520777474732066726D20686F20
:102470006D656D616465207478203D20676C207700
:102480006964207572206177617264203D206D6EF1
:10249000692073746E732066726D20646C20776C93
:1024A0002063616C6C20696E207465737420746D98
:1024B00077203D3D3B00646A316A77206465206483
:1024C0006C326B7467203D206761206C6272206FF4
:1024D0006D2073746566616E20657320746E78205C
:1024E0006665722063616C6C203D2075722072738A
:1024F000742069732035393920356E6E206573205C
:102500007566622073696773203D206D7920717450
:1025100068206973207374757474676172742073B2
:102520007475747467617274203D206E616D6520EE
:10253000616E647265617320616E6472656173209F
:102540003D20687065206F6B3F20646A316A772098
:10255000646520646C316B746720707365206B3B1D
:1025600000646B316F7420646520646D347A746626
:10257000203D2068616C6C6F206C6965626572201B
:1025800072616C66203D207363686F656E2C206DF0
:10259000616C2077696564657220766F6E2064696E
:1025A00072207A7520686F6572656E203D206973B0
:1025B0007420616C6C6573206F6B61792062656952
:1025C00020657563683F20776173206D616368746F
:1025D000206469652078796C3F2077697220747275
:1025E000656666656E20756E73206E6165636873DF
:1025F000746520776F636865207A756D2066642C3A
:10260000206B6F6D6D742069687220617563683F1F
:1026100020646B316F6220646520646D347A746667
:1026200020707365206B3B006737756E20646520F2
:10263000646C33727462203D206765206472206F81
:102640007020657820746E7820666572207572201F
:102650007270727420353939203D20757220727382
:10266000742069732035393920356E6E20746F6F90
:10267000203D20796F7572206B3320697320756659
:1026800062203D206D79207269672069732069633B
:102690006F6D20373630302069636F6D20373630EC
:1026A00030207077722031747420777474732061D5
:1026B0006E74203320656C206265616D203D207151
:1026C0007468206D756E696368206D756E696368E6
:1026D000203D206737756E20646520646C3372740A
:1026E0006220707365206B3B00646A366B626C20FD
:1026F000646520646C387A706C203D2068616C6C75
:102700006F206469657465722C207669656C656EEE
:102710002064616E6B2066756572206465696E6504
:102720006E207270727420353739203D206D6569D6
:102730006E20756D7A756720696E73206E6575659C
:10274000207174682069737420696E203220776F5D
:102750006368656E203D2069636820686F66666502
:102760002C206461737320646572206D6173742022
:102770006E616563687374657320776F6368656EF7
:10278000656E646520617566676562617574207742
:10279000697264203D20373320756E64206269734E
:1027A000207A756D206E616563687374656E206F45
:1027B00076206162656E64203D20646A366B626CCF
:1027C00020646520646C387A706C20707365206BAF
:1027D0003B006467367472206465206C61316173FC
:1027E000203D20746E7820666572207270727420AD
:1027F000647220616E6472656173203D206D792082
:102800007269672069732061206B656E776F6F64F2
:10281000207473353930207473353930203D207081
:102820007772206E7720353020777474732035747A
:102830002077747473203D20616E74206973206763
:102840003572762067357276203D20777820657264
:102850006520697320736E6F772061627420312068
:1028600063203D206D6E6920746E7820666572204D
:1028700071736F203D2071736C206F6B20766961DE
:1028800020627572656175203D20707365206B3B19
:1028900000646C3161626320646520646B356C7424
:1028A00072203D206761206C6272206F6D206A6F1C
:1028B000616368696D203D206861626520766F6E96
:1028C000206465696E656D206572666F6C67206255
:1028D00065696D206B6F6E74657374206765686FD2
:1028E0006572742C20636F6E6772617473203D2073
:1028F00062697374206475206E61656368737465C2
:1029000020776F636865206175662064656D206659
:1029100069656C6464617920766F6D206F762064E0
:10292000616265693F2069636820777565657264D7
:1029300065206D6963682066726575656E203D3D32
:102940003B006466376B627620646520646C386691
:102950007767203D20737269206C6272206F6D2052
:102960006672616E7A203D20727374203332392092
:10297000333239203D2064657220737475726D2086
:102980006C65747A746520776F636865206861741C
:10299000206D65696E6520616E74656E6E6520627E
:1029A00065736368616564696774203D20696D20A3
:1029B0006D6F6D656E74206B616E6E20696368204B
:1029C0006E7572206D6974206469706F6C20756E0D
:1029D0006420313020777474732073656E64656E83
:1029E000203D20686F6666652C206475206B616EE3
:1029F0006E7374206D69636820656D7066616E67C3
:102A0000656E3F20707365206B3B00646C396464B5
:102A100071206465207061317771203D20676520E9
:102A20006472206F6D2074686F6D61732065732010
:102A3000746E78206665722063616C6C203D206442
:102A400065696E20727374206973203539392035B9
:102A50007474203D20717468206973206E65617202
:102A600020726F65726D6F6E6420726F65726D6F2C
:102A70006E64203D206E616D652069732070686909
:102A80006C207068696C203D207269672069732032
:102A90007961657375206674323030302066743227
:102AA00030303020707772206E7720383020777485
:102AB0007473203D206F6B3F20646C396464712017
:102AC000646520706131777120707365206B3B0005
:102AD000646C326B626420646520646A336B6B7073
:102AE000203D206E65696E206265726E642C2064E4
:102AF00075206769627374206E6F636820696D6DFD
:102B0000657220736F207363686C656368742077E7
:102B100069652064616D616C73203D207669656C28
:102B20006C65696368742077616572652073736290
:102B300020656865722065747761732066756572BB
:102B400020646963683F206869203D20646C326BB3
:102B5000626420646520646A336B6B7020707365F7
:102B6000206B3B00646C3369666120646520646B94
:102B70003976667A203D206774206F6D206D617212
:102B800074696E203D20646B2066657220727566E4
:102B9000203D2075722035393920356E6E20696EE2
:102BA000206B656C6B6865696D206B656C6B686527
:102BB000696D203D20646F6B2066323720663237A6
:102BC000203D206E616D6520776F6C6667616E6772
:102BD00020776F6C6667616E67203D2064652064B6
:102BE0006B3976667A20707365206B3B00646130C8
:102BF0006161206465206462397A7A203D207566BF
:102C00006220647220667264203D207073652075B6
:102C1000722071736C20776964207361652065731D
:102C2000203220697263207669612064697265636D
:102C30007420657320737572652063666D207377E9
:102C40006C207270727473203D20746E78206665FB
:102C5000722071736F2065732068706520637561E1
:102C6000676E20736E203D20646130616120646571
:102C7000206462397A7A20707365206B3B00646748
:102C8000386B637220646520646D316F676B203D23
:102C9000206E65696E206C6272206A616E206963C5
:102CA000682068616265206E6F6368206E69636882
:102CB000747320766F6E206465696E656D206E6535
:102CC00075656E20717468206765736568656E2030
:102CD0003D2073746568742064656E6E2064656958
:102CE0006E6520616E74656E6E65207363686F6ECD
:102CF0003F2064616E6E206B6F6D6D652069636847
:102D0000206D6F7267656E206D616C20766F7262E8
:102D10006569203D206467386B63722064652064B8
:102D20006D316F676B20707365206B3B00646C3294
:102D3000616C6120646520646B37766A76203D2083
:102D400070736520717270203D2077697220776FF3
:102D5000686E656E203130206B6D20656E7466651F
:102D6000726E742C20646120627261756368737482
:102D7000206475206B65696E652037353020777467
:102D80007473203D20696368206B616E6E206469F6
:102D90006368206C61757420756E64206465757459
:102DA0006C69636820686F6572656E203D20646C95
:102DB00032616C6120646520646B377676207073B5
:102DC00065206B3B00646C396B6B75206465206417
:102DD0006C35746577203D2068616C6C6F206C6287
:102DE000722072616C66203D206861737420647586
:102DF000206465696E656E206B3220656E646C6957
:102E00006368206665727469673F206B6C696E67E2
:102E10007420677574203D20727374203537392013
:102E200035376E203D206D65696E6520616E746575
:102E30006E6E65206973742065696E203420656C40
:102E4000206265616D203D20707772206162742080
:102E50003230302077747473203D20616C6C206FA9
:102E60006B3F20707365206B203D3D3B00521BE99A
:102E70001B791C071D8D1D231EDD1E6B1F0620B632
:102E8000204621D421B2223523C4232E24B6246126
:102E9000252826E926D227912842290B2AD02A6400
:102EA0002BED2B7E2C2D2DC52D02000000002400C3
:102EB00027002A0000000000250028002B00000049
:102EC0000000230026002900040404040404040470
:102ED00002020202020203030303030301020408C5
:102EE0001020408001020408102001020408102074
:102EF00000000007000201000003040600000000BB
:102F0000000000001618EA3111241FBECFEFD8E0F0
:102F1000DEBFCDBF14E0A0E0B1E0E2E0FEE602C01B
:102F200005900D92A23FB107D9F715E0A2EFB4E0EA
:102F300001C01D92AA3DB107E1F71FE2C8E0DFE240
:102F400004C02297FE010E94C436C430D107C9F7DD
:102F50000E9424320C94FF360C940000A0E0B0E0F4
:102F6000E4EBF7E10C94D036EC01A880B980CA807C
:102F7000DB80A114B104C104D10441F484E2A82E81
:102F800089EDB82E8BE5C82E87E0D82EC601B50195
:102F90002DE133EF41E050E00E94933627EA31E41F
:102FA00040E050E00E943F367B018C01C601B50134
:102FB0002DE133EF41E050E00E949336CA01B901A0
:102FC0002CEE34EF4FEF5FEF0E943F366E0D7F1D0A
:102FD000801F911F97FF04C061507040804090484F
:102FE000688379838A839B839B01AC015F77B901F6
:102FF000CA01CDB7DEB7EAE00C94EC360E94AE17FA
:1030000008958FE093E00E94AE17089560930F0338
:103010007093100380931103909312030895FB01A2
:10302000DC0105900D920020E1F70895CF92EF9218
:103030000F9382EF94E06CE04BE025E004E073E056
:10304000E72E52E0C52E0E94CD2E2091150330911F
:1030500016033093060520930505C901880F991FB3
:10306000820F931F90930805809307050F91EF90AF
:10307000CF900895CF93DF938091090590910A0531
:10308000892BA9F0C0E0D0E00BC0609105057091DC
:103090000605882777FD8095982F0E945D2F219641
:1030A0008091090590910A05C817D90774F36091BA
:1030B000050570910605660F771F882777FD8095B7
:1030C000982F0E945D2FDF91CF9108956091170393
:1030D000709118038091130320E030E040E050E04D
:1030E0000E94E1336091070570910805882777FDFC
:1030F0008095982F0E945D2F809113030E946E335C
:103100006091050570910605882777FD8095982FB9
:103110000E945D2F089560911703709118038091AC
:10312000130320E030E040E050E00E94E133609182
:10313000050570910605882777FD8095982F0E94D8
:103140005D2F809113030E946E336091050570918D
:103150000605882777FD8095982F0E945D2F08959A
:10316000809113036CED75E020E030E040E050E02A
:103170000E94E13362E370E080E090E00E945D2F06
:10318000809113030E946E3308951F93182F60914E
:103190002105709122056F5F7F4F70932205609328
:1031A000210582EF94E041E00E94E02D809121050D
:1031B000909122054097B4F082EF94E060E041E006
:1031C0000E94E02D82EF94E060E071E00E946232A4
:1031D00082EF94E060E041E00E94E02D1092220531
:1031E0001092210582EF94E0612F0E94CE2D1F9155
:1031F00008952091050530910605B901660F771FE6
:10320000620F731F660F771F882777FD8095982FB1
:103210000E945D2F80E20E94C5180895992787FDBE
:103220009095A92FB92FFC01B097EB35F10508F067
:10323000F0C1EC5CFF4FEE0FFF1F0590F491E02D05
:1032400009940E948B180E9466180E943A1881E423
:10325000DBC10E9466180E948B180E948B180E9486
:103260008B180E943A1882E4CFC10E9466180E940F
:103270008B180E9466180E948B180E943A1883E4EB
:10328000C3C10E9466180E948B180E948B180E946E
:103290003A1884E4B9C10E948B180E943A1885E458
:1032A000B3C10E948B180E948B180E9466180E945E
:1032B0008B180E943A1886E4A7C10E9466180E94E3
:1032C00066180E948B180E943A1887E49DC10E94DC
:1032D0008B180E948B180E948B180E948B180E94DA
:1032E0003A1888E491C10E948B180E948B180E94A2
:1032F0003A1889E489C10E948B180E9466180E94BE
:1033000066180E9466180E943A188AE47DC10E94DD
:1033100066180E948B180E9466180E943A188BE467
:1033200073C10E948B180E9466180E948B180E941D
:103330008B180E943A188CE467C10E9466180E949C
:1033400066180E943A188DE45FC10E9466180E94B8
:103350008B180E943A188EE457C10E9466180E948A
:1033600066180E9466180E943A188FE44DC10E94A8
:103370008B180E9466180E9466180E948B180E9483
:103380003A1880E541C10E9466180E9466180E94A2
:103390008B180E9466180E943A1881E535C10E9478
:1033A0008B180E9466180E948B180E943A1882E5BA
:1033B0002BC10E948B180E948B180E948B180E94B0
:1033C0003A1883E521C10E9466180E943A1884E5E4
:1033D0001BC10E948B180E948B180E9466180E94C5
:1033E0003A1885E511C10E948B180E948B180E9423
:1033F0008B180E9466180E943A1886E505C10E9443
:103400008B180E9466180E9466180E943A1887E579
:10341000FBC00E9466180E948B180E948B180E94A5
:1034200066180E943A1888E5EFC00E9466180E944C
:103430008B180E9466180E9466180E943A1889E547
:10344000E3C00E9466180E9466180E948B180E94B2
:103450008B180E943A188AE5D7C00E948B180E94E8
:1034600066180E9466180E9466180E9466180E94DC
:103470003A1881E3C9C00E948B180E948B180E94E1
:1034800066180E9466180E9466180E943A1882E325
:10349000BBC00E948B180E948B180E948B180E9440
:1034A00066180E9466180E943A1883E3ADC00E9415
:1034B0008B180E948B180E948B180E948B180E94F8
:1034C00066180E943A1884E39FC00E948B180E94DD
:1034D0008B180E948B180E948B180E948B180E94D8
:1034E0003A1885E391C00E9466180E948B180E94CA
:1034F0008B180E948B180E948B180E943A1886E342
:1035000083C00E9466180E9466180E948B180E9451
:103510008B180E948B180E943A1887E375C00E948E
:1035200066180E9466180E9466180E948B180E94F6
:103530008B180E943A1888E367C00E9466180E94A0
:1035400066180E9466180E9466180E948B180E94D6
:103550003A1889E359C00E9466180E9466180E94B2
:1035600066180E9466180E9466180E943A1880E346
:103570004BC00E9466180E9466180E948B180E9419
:103580008B180E9466180E9466180E943A188EE2F4
:103590003BC00E9466180E948B180E948B180E94E4
:1035A0008B180E9466180E943A188DE32DC00E9465
:1035B00066180E948B180E948B180E9466180E9441
:1035C0008B180E943A188FE21FC00E948B180E942D
:1035D0008B180E9466180E9466180E948B180E9421
:1035E0008B180E943A188FE30FC00E9466180E9441
:1035F00066180E948B180E948B180E9466180E9401
:1036000066180E943A188CE20E94C51808950E941C
:10361000F9180895DF92EF92FF920F931F93CF93C3
:10362000DF937C0100E010E0BBE3DB2E2FC0809134
:103630001D0390911E03019749F461E670E080E05C
:1036400090E025E830E040E050E008C061E670E03E
:1036500080E090E02BE730E040E050E00E94193637
:1036600068836B3771051CF06B5470406883862F3C
:103670000E940E19219685E0CF31D807C1F6D88275
:103680000E94F9180E94F9180F5F1F4F0E151F05B1
:103690001CF4CAE1D5E0CBCFDF91CF911F910F9100
:1036A000FF90EF90DF900895AF92BF92CF92DF929C
:1036B000EF92FF920F931F93CF93DF935C0161E032
:1036C00070E080E090E02DE330E040E050E00E94C8
:1036D0001936EB01CC0FDD1FCC0FDD1FC60FD71F36
:1036E000CB5DDC4FEE24FF2488818B3371F00E9488
:1036F0000E19F501EE0DFF1D899180830894E11CE0
:10370000F11C85E0E816F10479F760E370E080E0F1
:1037100090E02AE330E040E050E00E941936162F96
:10372000862F0E940E19E501CE0DDF1D188361E67C
:1037300070E080E090E02BE730E040E050E00E9455
:103740001936162F862F0E940E19198361E670E034
:1037500080E090E02BE730E040E050E00E94193636
:10376000162F862F0E940E191A83E3E0F0E0EE0E6A
:10377000FF1E6501CE0CDF1C8DEF9FEFE80EF91EDA
:103780000BE3F601008360E070E080E090E022E06F
:1037900030E040E050E00E9419366130710581054B
:1037A0009105A1F461E670E080E090E02BE730E065
:1037B00040E050E00E941936162F862F0E940E1905
:1037C000F60110830C830894E11CF11C61E070E0A9
:1037D00080E090E029E030E040E050E00E941936BF
:1037E000653071058105910589F48FE20E940E19FB
:1037F00085010E0D1F1D8FE2F801838380E70E9473
:103800000E1980E7F80184838BE385830E94F91801
:10381000DF91CF911F910F91FF90EF90DF90CF90AC
:10382000BF90AF9008950F931F93CF93DF938C01B8
:10383000C0E0D0E0F801EC0FFD1F80818B3339F43C
:1038400080912005882351F40E94F91807C00E9436
:103850000E19219681E0C030D80761F7DF91CF9132
:103860001F910F910895CF92DF92EF92FF920F93E5
:103870001F93CF93DF936B0121E020932005C0E0DD
:10388000D0E001967C010027F7FC0095102F24C0A2
:1038900060E070E080E090E0A80197010E94193696
:1038A0009B01220F331F260F371FC9018F5A9B4FD1
:1038B0000E94131C61E070E080E090E026E030E0C0
:1038C00040E050E00E941936643071058105910591
:1038D00011F40E94F9182196CC15DD05CCF2109256
:1038E0002005DF91CF911F910F91FF90EF90DF9016
:1038F000CF9008950F931F93DF93CF93CDB7DEB78B
:10390000C050D1400FB6F894DEBF0FBECDBFFC0152
:10391000EE0FFF1FE359F14D659174918E010F5F1A
:103920001F4FC8010E940F18C8010E94131C0E945B
:10393000F918C050DF4F0FB6F894DEBF0FBECDBFF1
:10394000CF91DF911F910F9108950F931F93DF93F4
:10395000CF93CDB7DEB76E970FB6F894DEBF0FBE2C
:10396000CDBFFC01EE0FFF1FEA5BF74E659174912E
:103970008E010F5F1F4FC8010E940F18C8010E94DF
:10398000131C0E94F9186E960FB6F894DEBF0FBE96
:10399000CDBFCF91DF911F910F9108950F931F938A
:1039A000DF93CF93CDB7DEB727970FB6F894DEBF7E
:1039B0000FBECDBFFC01EE0FFF1FE85AF74F659118
:1039C00074918E010F5F1F4FC8010E940F18C8012C
:1039D0000E94131C0E94F91827960FB6F894DEBFB8
:1039E0000FBECDBFCF91DF911F910F9108950F931F
:1039F0001F93DF93CF9300D000D000D0CDB7DEB7B8
:103A0000FC01EE0FFF1FE851FB4F659174918E0191
:103A10000F5F1F4FC8010E940F18C8010E94131C9E
:103A20000E94F91826960FB6F894DEBF0FBECDBFE0
:103A3000CF91DF911F910F9108950F931F93DF9303
:103A4000CF9300D000D00F92CDB7DEB7FC01EE0FC0
:103A5000FF1FEA5CFD4F659174918E010F5F1F4F50
:103A6000C8010E940F18C8010E94131C0E94F91877
:103A70000F900F900F900F900F90CF91DF911F91AB
:103A80000F910895DF92EF92FF920F931F938C0195
:103A900064E2E62E65E0F62EC701B8010E94022F0F
:103AA000D82E0F5F1F4FC701B8010E94022F382F79
:103AB00020E02D0D311DC9011F910F91FF90EF9056
:103AC000DF90089580E090E00E94421D90931A03D9
:103AD0008093190382E090E00E94421D90931803A6
:103AE0008093170384E090E00E94421D90931C0392
:103AF00080931B0386E090E00E94421D90930A058C
:103B00008093090588E090E00E94421D9093200375
:103B100080931F038AE090E00E94421D909314035B
:103B2000809313038CE090E00E94421D90930C055B
:103B300080930B058EE090E00E94421D90931E033F
:103B400080931D0380E190E00E94421D909319052F
:103B50008093180508950F931F930E94621D809112
:103B6000130361E00E941D3086E060E00E941D307A
:103B700086E061E00E94433088E060E00E941D30F2
:103B800088E061E00E94433087E060E00E941D30E1
:103B900087E061E00E94433082EB95E040E855E227
:103BA00060E070E00E941F3180E00E94FB2F0E94C5
:103BB000373602EF14E0C80160E142E020E00E94E5
:103BC000172EC80161E171E00E946232C8016DE107
:103BD00071E00E946232C80160E041E00E94E02D85
:103BE000C80163E271E00E94623264EC79E080E037
:103BF00090E00E945D2FC8010E940F2E6091190372
:103C000070911A0380EB94E00E945E36CB017093B2
:103C100016036093150370930605609305059B01D9
:103C2000220F331F280F391F3093080520930705F3
:103C30001F910F910895DF92EF92FF920F931F93C0
:103C40008C01462FD72EE4E2EE2EE5E0FE2EC701D2
:103C5000B8010E94092F0F5F1F4FC701B8014D2DFA
:103C60000E94092F1F910F91FF90EF90DF90089510
:103C70000F931F93CF93DF9382EF94E00E940F2E58
:103C800082EF94E060E040E00E94E02D82EF94E05B
:103C900065E371E00E94623286E00E949B30892BCE
:103CA000C9F48091230390912403019690932403F7
:103CB00080932303099744F081E090E090932403DC
:103CC000809323030E94B01868EC70E080E090E0DD
:103CD0000E945D2F88E00E949B30892BC1F4809167
:103CE000230390912403019790932403809323034B
:103CF0001816190634F088E090E09093240380931E
:103D0000230368EC70E080E090E00E945D2F87E084
:103D10000E949B30892B11F010E007C068EC70E026
:103D200080E090E00E945D2F11E08091230390914C
:103D300024038430910509F4C0C28530910564F4F0
:103D40008230910509F40CC1833091050CF0DEC17D
:103D5000019709F029C610C08630910509F420C4E6
:103D6000863091050CF47CC38730910509F4A7C413
:103D7000089709F019C632C582EF94E060E041E08F
:103D80000E94E02D82EF94E06CE371E00E946232C9
:103D9000113009F0BFC082EF94E00E940F2E82EF35
:103DA00094E060E040E00E94E02D82EF94E06CE35C
:103DB00071E00E94623282EF94E060E041E00E9494
:103DC000E02D82EF94E06CE471E00E94623282EFB9
:103DD00094E06CE041E00E94E02D60911903709145
:103DE0001A0382EF94E04AE050E00E943A3366E919
:103DF00070E080E090E00E945D2FCCE3D0E086E0B0
:103E00000E949B30892B79F58091190390911A03B8
:103E1000019690931A038093190368EC70E080E098
:103E200090E00E945D2F8091190390911A03CD9725
:103E300024F0D0931A03C093190382EF94E069E54C
:103E400071E00E94623282EF94E06CE041E00E94F7
:103E5000E02D6091190370911A0382EF94E04AE01B
:103E600050E00E943A3388E00E949B30892B89F50C
:103E70008091190390911A03019790931A038093EC
:103E8000190368EC70E080E090E00E945D2F809163
:103E9000190390911A030A9734F48AE090E0909302
:103EA0001A038093190382EF94E069E571E00E94A0
:103EB000623282EF94E06CE041E00E94E02D60917C
:103EC000190370911A0382EF94E04AE050E00E94D7
:103ED0003A3387E00E949B30892B09F090CF82EF24
:103EE00094E060E041E00E94E02D82EF94E060E029
:103EF00071E00E94623282EF94E060E041E00E9453
:103F0000E02D64E670E080E090E00E945D2F81E0AB
:103F1000809323051092220510922105E091190348
:103F2000F0911A0380EB94E0BF010E945E3660932B
:103F30001503709316036093050570930605209191
:103F4000150330911603C901880F991F820F931F23
:103F5000909308058093070580E090E0BF0122C59B
:103F600082EF94E060E041E00E94E02D82EF94E077
:103F70006CE571E00E946232112309F4C0C082EF47
:103F800094E00E940F2E82EF94E060E040E00E94F7
:103F9000E02D82EF94E06CE571E00E94623282EFE6
:103FA00094E060E041E00E94E02D82EF94E068E65A
:103FB00071E00E94623282EF94E06AE041E00E9488
:103FC000E02D60911B0370911C0382EF94E04AE0A6
:103FD00050E00E943A3366E970E080E090E00E9491
:103FE0005D2F04EF11E0C9E1D0E086E00E949B3034
:103FF000892B81F580911B0390911C034996909326
:104000001C0380931B0368EC70E080E090E00E944A
:104010005D2F80911B0390911C03855F914024F0DC
:1040200010931C0300931B0382EF94E069E571E099
:104030000E94623282EF94E06AE041E00E94E02D4B
:1040400060911B0370911C0382EF94E04AE050E002
:104050000E943A3388E00E949B30892B79F5809149
:104060001B0390911C03499790931C0380931B039F
:1040700068EC70E080E090E00E945D2F80911B036F
:1040800090911C03499724F4D0931C03C0931B0305
:1040900082EF94E069E571E00E94623282EF94E081
:1040A0006AE041E00E94E02D60911B0370911C03C7
:1040B00082EF94E04AE050E00E943A3387E00E94A9
:1040C0009B30892B09F091CF82EF94E060E041E0D2
:1040D0000E94E02D82EF94E060E071E00E94623285
:1040E00082EF94E060E041E00E94E02D64E670E041
:1040F00080E090E00E945D2F81E080932305609135
:104100001B0370911C0384E090E04CC482EF94E0A8
:1041100060E041E00E94E02D82EF94E062E771E010
:104120000E946232112309F4C1C082EF94E00E9420
:104130000F2E82EF94E060E040E00E94E02D82EFDD
:1041400094E06BE771E00E94623282EF94E060E0FD
:1041500041E00E94E02D82EF94E069E871E00E9466
:10416000623282EF94E06AE041E00E94E02D6091CB
:1041700017037091180382EF94E04AE050E00E9428
:104180003A3366E970E080E090E00E945D2F00EB3A
:1041900014E0C4EFD1E086E00E949B30892B81F5CA
:1041A0008091170390911803C296909318038093FF
:1041B000170368EC70E080E090E00E945D2F809132
:1041C000170390911803815B944024F01093180317
:1041D0000093170382EF94E069E571E00E94623278
:1041E00082EF94E06AE041E00E94E02D60911703C5
:1041F0007091180382EF94E04AE050E00E943A3355
:1042000088E00E949B30892B81F580911703909163
:104210001803C297909318038093170368EC70E01B
:1042200080E090E00E945D2F809117039091180329
:10423000845F914024F4D0931803C093170382EF56
:1042400094E069E571E00E94623282EF94E06AE0F6
:1042500041E00E94E02D609117037091180382EFF6
:1042600094E04AE050E00E943A3387E00E949B309D
:10427000892B09F090CF82EF94E060E041E00E944A
:10428000E02D82EF94E060E071E00E94623282EF04
:1042900094E060E041E00E94E02D64E670E080E0A0
:1042A00090E00E945D2F81E08093230560911703C9
:1042B0007091180382E090E075C382EF94E060E0B3
:1042C00041E00E94E02D82EF94E063E971E00E94FA
:1042D0006232112309F4BDC082EF94E00E940F2ED8
:1042E00082EF94E060E040E00E94E02D82EF94E0F5
:1042F00063E971E00E94623282EF94E060E041E0A5
:104300000E94E02D82EF94E06EE971E00E9462323B
:1043100082EF94E066E041E00E94E02D60910905A3
:1043200070910A0582EF94E04AE050E00E943A332F
:1043300066E970E080E090E00E945D2FC9E0D0E087
:1043400086E00E949B30892B79F580910905909138
:104350000A05019690930A058093090568EC70E0C0
:1043600080E090E00E945D2F8091090590910A0500
:104370000A9724F0D0930A05C093090582EF94E0D0
:1043800069E571E00E94623282EF94E066E041E00C
:104390000E94E02D6091090570910A0582EF94E07A
:1043A0004AE050E00E943A3388E00E949B30892B1B
:1043B00079F58091090590910A05019790930A0576
:1043C0008093090568EC70E080E090E00E945D2F2A
:1043D0008091090590910A0597FF04C010920A0583
:1043E0001092090582EF94E069E571E00E94623263
:1043F00082EF94E066E041E00E94E02D60910905C3
:1044000070910A0582EF94E04AE050E00E943A334E
:1044100087E00E949B30892B09F092CF82EF94E0D5
:1044200060E041E00E94E02D82EF94E060E071E006
:104430000E94623282EF94E060E041E00E94E02D51
:1044400064E670E080E090E00E945D2F81E0809360
:1044500023056091090570910A0586E090E0A2C2EB
:1044600082EF94E060E041E00E94E02D82EF94E072
:1044700064EA71E00E946232112309F47BC082EF8A
:1044800094E00E940F2E82EF94E060E040E00E94F2
:10449000E02D82EF94E064EA71E00E94623282EFE4
:1044A00094E060E041E00E94E02D80911303909140
:1044B00014030D9729F482EF94E06CEA71E004C0D4
:1044C00082EF94E06AEB71E00E94623266E970E08C
:1044D00080E090E00E945D2F09E010E0CDE0D0E0A8
:1044E00086E00E949B30892B81F482EF94E060E0AB
:1044F00041E00E94E02D82EF94E06AEB71E00E94BF
:104500006232109314030093130388E00E949B30DF
:10451000892B81F482EF94E060E041E00E94E02D7D
:1045200082EF94E06CEA71E00E946232D09314034F
:10453000C093130387E00E949B30892B89F682EF9A
:1045400094E060E041E00E94E02D82EF94E060E0C2
:1045500071E00E94623282EF94E060E041E00E94EC
:10456000E02D64E670E080E090E00E945D2F81E045
:104570008093230560911303709114038AE090E007
:104580000E941B1E8DE060E00E941D3089E060E00B
:104590000E941D308091130361E00E941D3004C20F
:1045A00082EF94E060E041E00E94E02D82EF94E031
:1045B00068EC71E00E946232112309F479C082EF45
:1045C00094E00E940F2E82EF94E060E040E00E94B1
:1045D000E02D82EF94E068EC71E00E94623282EF9D
:1045E00094E060E041E00E94E02D80910B05909105
:1045F0000C05892B29F482EF94E063ED71E004C08F
:1046000082EF94E06EED71E00E94623266E970E044
:1046100080E090E00E945D2FC1E0D0E088E00E9441
:104620009B30892B81F482EF94E060E041E00E94AE
:10463000E02D82EF94E063ED71E00E94623210920F
:104640000C0510920B0586E00E949B30892B81F4AB
:1046500082EF94E060E041E00E94E02D82EF94E080
:104660006EED71E00E946232D0930C05C0930B0591
:1046700087E00E949B30892B89F682EF94E060E00E
:1046800041E00E94E02D82EF94E060E071E00E9442
:10469000623282EF94E060E041E00E94E02D64E647
:1046A00070E080E090E00E945D2F81E08093230520
:1046B00060910B0570910C058CE090E073C182EF66
:1046C00094E060E041E00E94E02D82EF94E069EE2A
:1046D00071E00E946232112309F479C082EF94E004
:1046E0000E940F2E82EF94E060E040E00E94E02DF7
:1046F00082EF94E069EE71E00E94623282EF94E012
:1047000060E041E00E94E02D80911D0390911E0326
:10471000892B29F482EF94E065EF71E004C082EF09
:1047200094E063E072E00E94623266E970E080E04B
:1047300090E00E945D2FC1E0D0E088E00E949B30B5
:10474000892B81F482EF94E060E041E00E94E02D4B
:1047500082EF94E065EF71E00E94623210921E03D6
:1047600010921D0386E00E949B30892B81F482EF1A
:1047700094E060E041E00E94E02D82EF94E063E08D
:1047800072E00E946232D0931E03C0931D0387E043
:104790000E949B30892B89F682EF94E060E041E033
:1047A0000E94E02D82EF94E060E071E00E946232AE
:1047B00082EF94E060E041E00E94E02D64E670E06A
:1047C00080E090E00E945D2F81E08093230560915E
:1047D0001D0370911E038EE090E0E4C082EF94E030
:1047E00060E041E00E94E02D82EF94E061E172E040
:1047F0000E946232113009F0CBC082EF94E00E9437
:104800000F2E82EF94E060E040E00E94E02D82EF06
:1048100094E061E172E00E94623282EF94E060E035
:1048200041E00E94E02D82EF94E06DE172E00E9491
:10483000623282EF94E06DE170E04AE050E00E9465
:104840003A3382EF94E065E272E00E94623282EFD6
:1048500094E06DE041E00E94E02D609118057091B8
:10486000190582EF94E04AE050E00E943A3366E98D
:1048700070E080E090E00E945D2FCDE1D0E086E026
:104880000E949B30892B79F580911805909119052C
:104890000196909319058093180568EC70E080E00C
:1048A00090E00E945D2F80911805909119054E9718
:1048B00024F0D0931905C093180582EF94E069E5C0
:1048C00071E00E94623282EF94E06DE041E00E946C
:1048D000E02D609118057091190582EF94E04AE08F
:1048E00050E00E943A3388E00E949B30892B79F592
:1048F000809118059091190501979093190580935F
:10490000180568EC70E080E090E00E945D2F8091D7
:1049100018059091190597FF04C01092190510927F
:10492000180582EF94E069E571E00E94623282EF3F
:1049300094E06DE041E00E94E02D609118057091D7
:10494000190582EF94E04AE050E00E943A3387E094
:104950000E949B30892B09F092CF82EF94E060E0B7
:1049600041E00E94E02D82EF94E060E071E00E945F
:10497000623282EF94E060E041E00E94E02D64E664
:1049800070E080E090E00E945D2F81E0809323053D
:104990001092220510922105609118057091190559
:1049A00080E190E00E941B1EDF91CF911F910F913B
:1049B0000895EF92FF920F931F93CF93DF9382EFAF
:1049C00094E00E940F2E82EF94E060E040E00E94AD
:1049D000E02D82EF94E068E272E00E94623286E0AD
:1049E0000E949B30892B99F480912103909122039E
:1049F000019690932203809321030B9744F081E06A
:104A000090E090932203809321030E94B01888E0E5
:104A10000E949B30892B91F4809121039091220375
:104A2000019790932203809321031816190634F0FE
:104A30008AE090E0909322038093210387E00E9414
:104A40009B30892B11F010E007C064E670E080E035
:104A500090E00E945D2F11E080912103909122034C
:104A60008530910509F42EC3863091059CF482307F
:104A7000910509F4EDC08330910524F4019709F004
:104A8000C7C71FC08330910509F444C1049709F0DA
:104A9000BFC72CC28830910509F4C6C5893091057D
:104AA00044F48630910509F4F9C3079709F0B0C7BB
:104AB000E1C48930910509F49AC60A9709F0A8C79C
:104AC00080C782EF94E060E041E00E94E02D82EF39
:104AD00094E064E372E00E946232113009F098C7FA
:104AE00082EF94E00E940F2E82EF94E060E040E0BD
:104AF0000E94E02D82EF94E061E472E00E94623255
:104B00001092220510922105C1E0D0E098C082EFFA
:104B100094E06CE040E00E94E02D82EF94E0BE0162
:104B20004AE050E00E943A3382EF94E061E0409125
:104B300021050E94E02D62E070E080E090E029E035
:104B400030E040E050E00E9419366230710579F49F
:104B500060E070E080E090E027E430E040E050E08A
:104B60000E941936DC01CB010E941D1D35C0633047
:104B7000710579F460E070E080E090E02FE630E0CD
:104B800040E050E00E941936DC01CB010E94F71C86
:104B900023C06430710579F460E070E080E090E05B
:104BA0002FE630E040E050E00E941936DC01CB01F6
:104BB0000E94CE1C11C06530710574F060E070E099
:104BC00080E090E027E831E040E050E00E941936B4
:104BD000DC01CB010E94A51C80912105909122054A
:104BE0000197909322058093210580910B05909168
:104BF0000C05019719F587E00E949B30892BD9F7A6
:104C00000E94B01868EE73E080E090E00E945D2F93
:104C100082EF94E060E041E00E94E02D82EF94E0BA
:104C200060E071E00E94623282EF94E060E041E077
:104C30000E94E02D1092220510922105219680916C
:104C40001B0390911C038C179D070CF060CFE0C6EE
:104C500082EF94E060E041E00E94E02D82EF94E07A
:104C600069E472E00E946232113009F0D1C682EF2D
:104C700094E00E940F2E82EF94E060E040E00E94FA
:104C8000E02D82EF94E066E572E00E9462321092BD
:104C900022051092210582EF94E06CE040E00E9432
:104CA000E02D809118059091190597FF04C010928E
:104CB000190510921805609118057091190582EF79
:104CC00094E04AE050E00E943A3382EF94E061E0E1
:104CD000409121050E94E02D8091180590911905C1
:104CE0000E947A1C80911805909119050196909365
:104CF0001905809318054E9724F01092190510920B
:104D00001805609118057091190580E190E00E94E6
:104D10001B1E7EC682EF94E060E041E00E94E02D21
:104D200082EF94E06FE572E00E946232113009F088
:104D30006FC682EF94E00E940F2E82EF94E060E055
:104D400040E00E94E02D82EF94E06FE672E00E9466
:104D50006232109222051092210501E010E0BDC0E0
:104D600082EF94E06CE040E00E94E02D82EF94E05E
:104D7000B8014AE050E00E943A3382EF94E060913B
:104D8000210541E00E94E02D60E070E080E090E0CD
:104D900026E430E040E050E00E941936DC01CB010F
:104DA0007C010E941D1D8091210590912205019793
:104DB000909322058093210580910B0590910C051D
:104DC000019709F088C0C0911903D0911A03249764
:104DD00041C086E00E949B30892B59F40E94B01894
:104DE00068EE73E080E090E00E945D2FC7010E94B2
:104DF0001D1D88E00E949B30892B31F50E94B01860
:104E000068EE73E080E090E00E945D2F80EB94E01C
:104E1000BE010E945E366093150370931603609383
:104E20000505709306052091150330911603C901FD
:104E3000880F991F820F931F909308058093070591
:104E4000C7010E941D1D249768EC70E080E090E08F
:104E50000E945D2F87E00E949B30892B09F0B9CF1B
:104E60000E94B01868EE73E080E090E00E945D2F31
:104E70006091190370911A0380EB94E00E945E36F2
:104E800060931503709316036093050570930605F0
:104E90002091150330911603C901880F991F820FC5
:104EA000931F909308058093070582EF94E060E0DC
:104EB00041E00E94E02D82EF94E060E071E00E940A
:104EC000623282EF94E060E041E00E94E02D1092B7
:104ED0002205109221050F5F1F4F80911B039091B7
:104EE0001C03801791070CF03BCF92C582EF94E032
:104EF00060E041E00E94E02D82EF94E06BE772E019
:104F00000E946232113009F083C582EF94E00E9462
:104F10000F2E82EF94E060E040E00E94E02D82EFEF
:104F200094E06BE872E00E946232109222051092C7
:104F3000210501E010E0BDC082EF94E06CE040E0AC
:104F40000E94E02D82EF94E0B8014AE050E00E9418
:104F50003A3382EF94E06091210541E00E94E02D18
:104F600060E070E080E090E02EE630E040E050E06D
:104F70000E941936DC01CB017C010E94F71C809154
:104F80002105909122050197909322058093210598
:104F900080910B0590910C05019709F088C0C09194
:104FA0001903D0911A03249741C086E00E949B30D8
:104FB000892B59F40E94B01868EE73E080E090E00D
:104FC0000E945D2FC7010E94F71C88E00E949B3061
:104FD000892B31F50E94B01868EE73E080E090E014
:104FE0000E945D2F80EB94E0BE010E945E366093CC
:104FF00015037093160360930505709306052091C1
:10500000150330911603C901880F991F820F931F52
:105010009093080580930705C7010E94F71C249709
:1050200068EC70E080E090E00E945D2F87E00E94D5
:105030009B30892B09F0B9CF0E94B01868EE73E05D
:1050400080E090E00E945D2F6091190370911A0337
:1050500080EB94E00E945E36609315037093160314
:105060006093050570930605209115033091160392
:10507000C901880F991F820F931F90930805809391
:10508000070582EF94E060E041E00E94E02D82EFAE
:1050900094E060E071E00E94623282EF94E060E0B0
:1050A00041E00E94E02D10922205109221050F5F31
:1050B0001F4F80911B0390911C03801791070CF0E8
:1050C0003BCFA6C482EF94E060E041E00E94E02D77
:1050D00082EF94E067E972E00E946232113009F0D9
:1050E00097C482EF94E00E940F2E82EF94E060E07C
:1050F00040E00E94E02D82EF94E067EA72E00E94B7
:105100006232109222051092210501E010E0BDC02C
:1051100082EF94E06CE040E00E94E02D82EF94E0AA
:10512000B8014AE050E00E943A3382EF94E0609187
:10513000210541E00E94E02D60E070E080E090E019
:105140002EE630E040E050E00E941936DC01CB0151
:105150007C010E94CE1C809121059091220501972F
:10516000909322058093210580910B0590910C0569
:10517000019709F088C0C0911903D0911A032497B0
:1051800041C086E00E949B30892B59F40E94B018E0
:1051900068EE73E080E090E00E945D2FC7010E94FE
:1051A000CE1C88E00E949B30892B31F50E94B018FC
:1051B00068EE73E080E090E00E945D2F80EB94E069
:1051C000BE010E945E3660931503709316036093D0
:1051D0000505709306052091150330911603C9014A
:1051E000880F991F820F931F9093080580930705DE
:1051F000C7010E94CE1C249768EC70E080E090E02C
:105200000E945D2F87E00E949B30892B09F0B9CF67
:105210000E94B01868EE73E080E090E00E945D2F7D
:105220006091190370911A0380EB94E00E945E363E
:10523000609315037093160360930505709306053C
:105240002091150330911603C901880F991F820F11
:10525000931F909308058093070582EF94E060E028
:1052600041E00E94E02D82EF94E060E071E00E9456
:10527000623282EF94E060E041E00E94E02D109203
:105280002205109221050F5F1F4F80911B03909103
:105290001C03801791070CF03BCFBAC382EF94E058
:1052A00060E041E00E94E02D82EF94E063EB72E069
:1052B0000E946232113009F0ABC382EF94E00E9489
:1052C0000F2E82EF94E060E040E00E94E02D82EF3C
:1052D00094E061E472E00E94623210922205109222
:1052E000210501E010E0BDC082EF94E06CE040E0F9
:1052F0000E94E02D82EF94E0B8014AE050E00E9465
:105300003A3382EF94E06091210541E00E94E02D64
:1053100060E070E080E090E026E831E040E050E0BE
:105320000E941936DC01CB017C010E94A51C8091F2
:1053300021059091220501979093220580932105E4
:1053400080910B0590910C05019709F088C0C091E0
:105350001903D0911A03249741C086E00E949B3024
:10536000892B59F40E94B01868EE73E080E090E059
:105370000E945D2FC7010E94A51C88E00E949B30FF
:10538000892B31F50E94B01868EE73E080E090E060
:105390000E945D2F80EB94E0BE010E945E36609318
:1053A000150370931603609305057093060520910D
:1053B000150330911603C901880F991F820F931F9F
:1053C0009093080580930705C7010E94A51C2497A8
:1053D00068EC70E080E090E00E945D2F87E00E9422
:1053E0009B30892B09F0B9CF0E94B01868EE73E0AA
:1053F00080E090E00E945D2F6091190370911A0384
:1054000080EB94E00E945E36609315037093160360
:1054100060930505709306052091150330911603DE
:10542000C901880F991F820F931F909308058093DD
:10543000070582EF94E060E041E00E94E02D82EFFA
:1054400094E060E071E00E94623282EF94E060E0FC
:1054500041E00E94E02D10922205109221050F5F7D
:105460001F4F80911B0390911C03801791070CF034
:105470003BCFCEC282EF94E060E041E00E94E02D9D
:1054800082EF94E062EC72E00E946232113009F027
:10549000BFC282EF94E00E940F2E82EF94E060E0A2
:1054A00040E00E94E02D82EF94E062EC72E00E9406
:1054B0006232109222051092210501E010E0ABC08B
:1054C00082EF94E06CE040E00E94E02D82EF94E0F7
:1054D000B8014AE050E00E943A3382EF94E06091D4
:1054E000210541E00E94E02D8DE095E00E94541BD3
:1054F00080910B0590910C05019709F08AC0C0912D
:105500001903D0911A03249743C086E00E949B3070
:10551000892B61F40E94B01868EE73E080E090E09F
:105520000E945D2F8DE095E00E94131C88E00E9490
:105530009B30892B39F50E94B01868EE73E080E04B
:1055400090E00E945D2F80EB94E0BE010E945E36E9
:105550006093150370931603609305057093060519
:105560002091150330911603C901880F991F820FEE
:10557000931F90930805809307058DE095E00E94A6
:10558000131C249768EC70E080E090E00E945D2F8F
:1055900087E00E949B30892B09F0B7CF0E94B0189A
:1055A00068EE73E080E090E00E945D2F6091190347
:1055B00070911A0380EB94E00E945E3660931503AD
:1055C00070931603609305057093060520911503EB
:1055D00030911603C901880F991F820F931F909372
:1055E00008058093070582EF94E060E041E00E94A7
:1055F000E02D82EF94E060E071E00E94623282EF81
:1056000094E060E041E00E94E02D109222051092AB
:1056100021050F5F1F4F80911B0390911C03801782
:1056200091070CF04DCFF4C182EF94E060E041E0CF
:105630000E94E02D82EF94E069EE71E00E946232F8
:10564000113009F0E5C182EF94E00E940F2E82EF45
:1056500094E060E040E00E94E02D82EF94E06DEC89
:1056600072E00E946232109222051092210501E040
:1056700010E0B4C082EF94E06CE040E00E94E02DC6
:1056800082EF94E0B8014AE050E00E943A3382EFA2
:1056900094E06091210541E00E94E02D81E090E0DE
:1056A0000E940A1B809121059091220501979093F9
:1056B00022058093210580910B0590910C0501979F
:1056C00009F08AC0C0911903D0911A03249743C0EE
:1056D00086E00E949B30892B61F40E94B01868EE2E
:1056E00073E080E090E00E945D2F8AE195E00E94E7
:1056F000131C88E00E949B30892B39F50E94B0185A
:1057000068EE73E080E090E00E945D2F80EB94E013
:10571000BE010E945E36609315037093160360937A
:105720000505709306052091150330911603C901F4
:10573000880F991F820F931F909308058093070588
:105740008AE195E00E94131C249768EC70E080E0E9
:1057500090E00E945D2F87E00E949B30892B09F02A
:10576000B7CF0E94B01868EE73E080E090E00E942E
:105770005D2F6091190370911A0380EB94E00E94F1
:105780005E3660931503709316036093050570935E
:1057900006052091150330911603C901880F991F42
:1057A000820F931F909308058093070582EF94E082
:1057B00060E041E00E94E02D82EF94E060E071E063
:1057C0000E94623282EF94E060E041E00E94E02DAE
:1057D00010922205109221050F5F1F4F80911B032D
:1057E00090911C03801791070CF044CF11C182EFF8
:1057F00094E060E041E00E94E02D82EF94E06AEDE9
:1058000072E00E946232113009F002C182EF94E02E
:105810000E940F2E82EF94E060E040E00E94E02DB5
:1058200082EF94E06AED72E00E94623282EF94E0CF
:1058300060E041E00E94E02D82EF94E067EE72E0CC
:105840000E94623282EF94E06AE041E00E94E02D23
:1058500060911F037091200382EF94E04AE050E0D2
:105860000E943A3366E970E080E090E00E945D2F8C
:1058700017E2E12EF12CC1E0D0E086E00E949B30DF
:10588000892B79F580911F039091200301969093C5
:10589000200380931F0368EC70E080E090E00E949A
:1058A0005D2F80911F0390912003889724F0F09240
:1058B0002003E0921F0382EF94E060EF72E00E9409
:1058C000623282EF94E06AE041E00E94E02D609154
:1058D0001F037091200382EF94E04AE050E00E94A1
:1058E0003A3388E00E949B30892B81F580911F0319
:1058F0009091200301979093200380931F0368ECFD
:1059000070E080E090E00E945D2F80911F039091F5
:1059100020031816190624F0D0932003C0931F0308
:1059200082EF94E060EF72E00E94623282EF94E0D6
:105930006AE041E00E94E02D60911F037091200316
:1059400082EF94E04AE050E00E943A3387E00E9400
:105950009B30892B11F010E013C082EF94E060E0DF
:1059600041E00E94E02D82EF94E064EF72E00E943B
:10597000623282EF94E060E041E00E94E02D11E0AD
:1059800060911F037091200388E090E00E941B1E2D
:10599000112309F472CF10922205109221058091F3
:1059A0001B0390911C03BC01660F771F660F771FC6
:1059B000680F791F80911F03909120030E94331C70
:1059C00027C082EF94E060E041E00E94E02D82EF8A
:1059D00094E069E073E00E946232113089F468EC6F
:1059E00070E080E090E006C00E94381E64E670E03F
:1059F00080E090E00E945D2F809123058823A1F331
:105A00001092230564E670E080E090E00E945D2F34
:105A1000DF91CF911F910F91FF90EF9008950E9419
:105A2000D92464EB70E080E090E00E945D2F08953F
:105A30000F931F938C01FC01848160E00E9443302E
:105A400081E090E00E94B62FF801848161E00E941D
:105A5000433081E090E00E94B62FF801848160E03D
:105A60000E94433084E690E00E94B62F1F910F9170
:105A70000895CF92DF92EF92FF920F931F93CF93EF
:105A8000DF93D82EC92E282F392FC9018C01C0E0F1
:105A9000D0E0E62EFF24F801858161E00E941D30F0
:105AA000B7010C2E02C0759567950A94E2F76170F4
:105AB000F80185810E94433021960F5F1F4FC83047
:105AC000D10549F78D2D9C2D0E94182DDF91CF9186
:105AD0001F910F91FF90EF90DF90CF900895CF929C
:105AE000DF92EF92FF920F931F93CF93DF93D82E05
:105AF000C92E282F392FC9018C01C0E0D0E0E62E35
:105B0000FF24F801858161E00E941D30B7010C2E51
:105B100002C0759567950A94E2F76170F801858176
:105B20000E94433021960F5F1F4FC430D10549F7C3
:105B30008D2D9C2D0E94182DDF91CF911F910F91DB
:105B4000FF90EF90DF90CF9008951F93CF93DF9356
:105B5000EC01162F8A81642F0E9443308B818F3F86
:105B600019F060E00E9443308D8584FF05C0CE01AE
:105B7000612F0E94392D0EC0612F70E084E0759571
:105B800067958A95E1F7CE010E946F2DCE01612FB6
:105B90000E946F2DDF91CF911F91089541E00E94E7
:105BA000A52D089540E00E94A52D0895FC0166856D
:105BB000862F846086876C60CF010E94D22D089565
:105BC000DF93CF93CDB7DEB728970FB6F894DEBF3B
:105BD0000FBECDBF9C01FE013196A8EDB4E088E078
:105BE0000D9001928150E1F7F9018189841710F439
:105BF000482F4150E42FF0E0EE0FFF1FEC0FFD1F88
:105C00008181680F6068C9010E94D22D28960FB665
:105C1000F894DEBF0FBECDBFCF91DF91089561E054
:105C20000E94D22D80ED97E00E94B62F0895CF9369
:105C3000DF93EC01423018F08D8588608D87498BA9
:105C40001A8A222329F0413019F48D8584608D87CA
:105C500080E593EC0E94B62F8A8160E00E94433079
:105C60008C8160E00E9443308B818F3F19F060E0AF
:105C70000E9443306D8564FD1DC0CE0163E00E942B
:105C80006F2D84E991E10E94B62FCE0163E00E945E
:105C90006F2D84E991E10E94B62FCE0163E00E944E
:105CA0006F2D86E990E00E94B62FCE0162E00E943F
:105CB0006F2D16C06062CE010E94D22D84E991E161
:105CC0000E94B62F6D856062CE010E94D22D86E9BA
:105CD00090E00E94B62F6D856062CE010E94D22DA9
:105CE0006D856062CE010E94D22D84E08E87CE0148
:105CF0000E94D62DCE010E940F2E82E08F87CE010A
:105D000066E00E94D22DDF91CF9108956F927F922D
:105D10008F92AF92CF92EF920F931F93DF93CF9317
:105D2000CDB7DEB73C01162F842FF30142832383C6
:105D30000483E582C682A78280869D8591879E85A1
:105D400092879F8593879889948761E00E941D3090
:105D5000F30183818F3F19F061E00E941D30F30150
:105D6000848161E00E941D30112319F0F301158632
:105D700003C080E1F3018587C30160E141E020E0D9
:105D80000E94172ECF91DF911F910F91EF90CF902E
:105D9000AF908F907F906F9008958F92AF92CF9237
:105DA000EF920F931F93CF93DF93DC01362F542F85
:105DB000722F102FAE2C8C2C82ED94E011969C93B8
:105DC0008E9300D000D0EDB7FEB73196CDB7DEB7D9
:105DD0001982118212821382CD0161E0432F2FEFCD
:105DE000052FE72EC12E0E94862E0F900F900F9048
:105DF0000F90DF91CF911F910F91EF90CF90AF90C7
:105E00008F900895F999FECF72BD61BDF89A80B563
:105E10000895F999FECF1FBA72BD61BD40BD0FB69E
:105E2000F894FA9AF99A0FBE08951F920F920FB63E
:105E30000F9211242F933F938F939F93AF93BF9310
:105E40008091290590912A05A0912B05B0912C05F0
:105E500030912D050196A11DB11D232F2D5F2D37EA
:105E600020F02D570196A11DB11D20932D05809383
:105E7000290590932A05A0932B05B0932C058091BA
:105E8000250590912605A0912705B091280501963A
:105E9000A11DB11D8093250590932605A09327058C
:105EA000B0932805BF91AF919F918F913F912F9112
:105EB0000F900FBE0F901F9018959B01AC017FB7FC
:105EC000F8948091250590912605A0912705B09121
:105ED000280566B5A89B05C06F3F19F00196A11D66
:105EE000B11D7FBFBA2FA92F982F8827860F911D2C
:105EF000A11DB11D62E0880F991FAA1FBB1F6A95E3
:105F0000D1F7BC012DC0FFB7F89480912505909181
:105F10002605A0912705B0912805E6B5A89B05C0E8
:105F2000EF3F19F00196A11DB11DFFBFBA2FA92F98
:105F3000982F88278E0F911DA11DB11DE2E0880FBB
:105F4000991FAA1FBB1FEA95D1F7861B970B885E86
:105F50009340C8F2215030404040504068517C4F3F
:105F6000211531054105510571F60895019739F064
:105F7000880F991F880F991F02970197F1F70895CD
:105F8000789484B5826084BD84B5816084BD85B514
:105F9000826085BD85B5816085BDEEE6F0E08081DB
:105FA00081608083E1E8F0E01082808182608083FC
:105FB000808181608083E0E8F0E08081816080837F
:105FC000E1EBF0E0808184608083E0EBF0E08081B1
:105FD00081608083EAE7F0E0808184608083808153
:105FE00082608083808181608083808180688083FB
:105FF0001092C1000895982F8E3008F09E5097702F
:106000008091CC048295880F880F807C892B8093A7
:106010007C0080917A00806480937A0080917A007D
:1060200086FDFCCF2091780040917900942F80E08C
:1060300030E0282B392BC9010895482F50E0CA01C0
:106040008452914DFC0124914853514DFA018491A1
:106050008823C1F0E82FF0E0EE0FFF1FE655F14D69
:10606000A591B491662341F49FB7F8948C91209543
:1060700082238C939FBF08959FB7F8948C91822BB5
:106080008C939FBF0895482F50E0CA018051914DD5
:10609000FC012491CA018452914DFC013491485372
:1060A000514DFA019491992309F444C0222351F1EE
:1060B000233071F0243028F42130A1F0223011F582
:1060C00014C02630B1F02730C1F02430D9F404C018
:1060D000809180008F7703C0809180008F7D8093B6
:1060E000800010C084B58F7702C084B58F7D84BDD9
:1060F00009C08091B0008F7703C08091B0008F7D80
:106100008093B000E92FF0E0EE0FFF1FEC54F14D4B
:10611000A591B491662341F49FB7F8948C91309582
:1061200083238C939FBF08959FB7F8948C91832B02
:106130008C939FBF0895682F70E0CB018051914DE3
:10614000FC012491CB018452914DFC014491685390
:10615000714DFB019491992319F420E030E03CC08B
:10616000222351F1233071F0243028F42130A1F0A2
:10617000223011F514C02630B1F02730C1F02430A0
:10618000D9F404C0809180008F7703C08091800093
:106190008F7D8093800010C084B58F7702C084B556
:1061A0008F7D84BD09C08091B0008F7703C080913E
:1061B000B0008F7D8093B000892F90E0880F991FE9
:1061C0008254914DFC01A591B4918C9120E030E076
:1061D000842311F021E030E0C90108951F920F924D
:1061E0000FB60F9211242F933F934F938F939F934A
:1061F000EF93FF934091C600E091AE05F091AF059B
:1062000031969F012F77307031978091B005909132
:10621000B1052817390739F0E25DFA4F4083309312
:10622000AF052093AE05FF91EF919F918F914F9114
:106230003F912F910F900FBE0F901F901895CF9305
:10624000DF93EC019A01AB01E885F985203081EEFE
:10625000380780E0480780E0580709F449C081E02A
:1062600090E00A8802C0880F991F0A94E2F78083A1
:1062700060E079E08DE390E00E9493362150304059
:1062800040405040CA01B90122E030E040E050E017
:106290000E949336EC81FD813083EE81FF81208363
:1062A000EA85FB85208141E050E0CA010E8402C0EE
:1062B000880F991F0A94E2F7282B2083EA85FB8533
:1062C0002081CA010F8402C0880F991F0A94E2F747
:1062D000282B2083EA85FB858081088802C0440F33
:1062E000551F0A94E2F7842B8083DF91CF910895A4
:1062F000108220E130E0CECFDC011296ED91FC91CE
:106300001397E058FF4F2191319180819181281B93
:10631000390B2F773070C9010895DC011296ED9189
:10632000FC911397EE57FF4F20813181929182911A
:10633000E058F0408217930719F42FEF3FEF05C0A4
:10634000E20FF31F8081282F30E0C9010895DC019E
:106350001296ED91FC911397DF01AE57BF4F2D912F
:106360003C911197E058FF4F80819181E058F040B7
:106370008217930719F42FEF3FEF0BC0E20FF31FC3
:1063800080812F5F3F4F2F7730702D933C93282FC4
:1063900030E0C9010895DC011296ED91FC9113974C
:1063A000EE57FF4F80819181929382930895FC0173
:1063B000A085B18521898C9190E0022E02C095952F
:1063C00087950A94E2F780FFF6CF0484F585E02DE7
:1063D0006083089584EE94E09093B3058093B205B2
:1063E0008EE295E09093B5058093B40585EC90E03E
:1063F0009093B7058093B60584EC90E09093B9052F
:106400008093B80580EC90E09093BB058093BA052B
:1064100081EC90E09093BD058093BC0586EC90E004
:106420009093BF058093BE0584E08093C00583E010
:106430008093C10587E08093C20585E08093C30502
:1064400081E08093C40508950E94C02F0E94AB1D77
:106450000E940F2DFDCF0F931F93CF93DF938C01DD
:10646000EB0109C02196D801ED91FC910190F081DA
:10647000E02DC801099568816623A1F7DF91CF91CE
:106480001F910F910895EF92FF920F931F93CF9357
:10649000DF938C017B01EA010CC0D7016D917D0176
:1064A000D801ED91FC910190F081E02DC801099592
:1064B0002197209791F7DF91CF911F910F91FF9036
:1064C000EF900895DC01ED91FC910280F381E02DC5
:1064D000099508952F923F924F925F926F927F920B
:1064E0008F929F92AF92BF92CF92DF92EF92FF92E4
:1064F0000F931F93DF93CF93CDB7DEB7A0970FB65F
:10650000F894DEBF0FBECDBF1C016A017B014115AF
:1065100051056105710549F440E350E060E070E029
:1065200020E030E00E94043356C0882499245401AE
:10653000422E55246624772401E010E00C0F1D1F25
:10654000080D191DC701B601A30192010E94713601
:10655000F80160830894811C911CA11CB11CC70127
:10656000B601A30192010E947136C901DA016C01E2
:106570007D01C114D104E104F104F1F681E0E82EBB
:10658000F12CEC0EFD1EE80CF91C3E010894611C78
:10659000711CD501C4010197A109B1096C01C8188A
:1065A000D90816C0F601EE0DFF1D40814A3010F4E7
:1065B000405D01C0495C552747FD5095652F752FFB
:1065C000C10120E030E00E9404330894E108F108A2
:1065D0006E147F0439F7A0960FB6F894DEBF0FBE95
:1065E000CDBFCF91DF911F910F91FF90EF90DF9082
:1065F000CF90BF90AF909F908F907F906F905F9063
:106600004F903F902F900895EF92FF920F931F931A
:10661000CF93DF93EC017A018B012115310541F411
:10662000E881F9810190F081E02D642F09951BC06C
:106630002A303105B1F477FF10C04DE250E060E040
:1066400070E020E030E00E94043310950095F09453
:10665000E094E11CF11C011D111DCE01B801A70140
:106660002AE00E946A32DF91CF911F910F91FF9033
:10667000EF900895EF92FF920F931F937B019A0181
:106680000027F7FC0095102FB801A7010E940433E2
:106690001F910F91FF90EF900895813041F081306C
:1066A00018F08230D1F409C010926E0008958091E4
:1066B0006F008D7F80936F000895809170008D7FB3
:1066C0008093700081E08093B0008091B100887F5A
:1066D00084608093B1001092B30008951F93182F27
:1066E0008091CD04811711F09FEF06C0E9EAFEE228
:1066F00094918FEF8093CD04892F0E944D33812F89
:1067000060E00E9443301F9108951F920F920FB6D0
:106710000F9211242F933F934F935F936F937F9327
:106720008F939F93AF93BF93EF93FF938091D30584
:106730009091D405A091D505B091D6050097A105FB
:10674000B10551F1E091D705F091D8058081909184
:10675000D905892780838091D3059091D405A09194
:10676000D505B091D605181619061A061B06C4F4ED
:106770008091D3059091D405A091D505B091D6050F
:106780000197A109B1098093D3059093D405A093F3
:10679000D505B093D60504C08091CD040E946E3318
:1067A000FF91EF91BF91AF919F918F917F916F91E9
:1067B0005F914F913F912F910F900FBE0F901F90BF
:1067C00018952F923F925F926F927F928F929F9235
:1067D000AF92BF92CF92DF92EF92FF920F931F93EF
:1067E000DF93CF9300D000D0CDB7DEB7A82F1B0129
:1067F00029833A834B835C838091CD048A1721F4EB
:10680000E9EAFEE2549082C08F3F09F0DAC1A0931A
:10681000CD04E9EAFEE254902FEF521609F4D1C1FB
:1068200081E0581639F192E0591609F449C0552013
:1068300009F06CC014BC15BC84B5826084BD85B5FC
:10684000816085BD2A2F30E0F901E853F14DE491D4
:10685000F0E0EE0FFF1FEC54F14D85919491909371
:10686000CA058093C9052452314DF9018491809362
:10687000CB054EC010928000109281008091810063
:106880008860809381008091810081608093810085
:106890002A2F30E0F901E853F14DE491F0E0EE0FDA
:1068A000FF1FEC54F14D859194919093D105809305
:1068B000D0052452314DF90184918093D20528C02E
:1068C0001092B0001092B1008091B000826080936D
:1068D000B0008091B10081608093B1002A2F30E038
:1068E000F901E853F14DE491F0E0EE0FFF1FEC5495
:1068F000F14D859194919093D8058093D7052452BA
:10690000314DF90184918093D90502C057FC59C1DA
:106910008A2F61E00E941D30552021F0F2E05F16C1
:1069200009F0BEC031018824992460E072E18AE751
:1069300090E0A40193010E94933659016A018601F7
:1069400075010894E108F108010911092FEFE21619
:10695000F1040105110509F008F499C060E472E43E
:106960008FE090E0A40193010E94933679018A019F
:106970000894E108F1080109110982E05816C1F4F0
:106980009FEFE916F1040105110509F008F484C030
:1069900060E970ED83E090E0A40193010E949336DA
:1069A00079018A010894E108F1080109110983E0DD
:1069B000AFEFEA16F1040105110509F008F468C00B
:1069C00068E478EE81E090E0A40193010E949336A0
:1069D00079018A010894E108F1080109110955209B
:1069E00011F483E01DC0B2E05B1611F084E018C022
:1069F000EFEFEE16F1040105110509F008F4DFC010
:106A000064E274EF80E090E0A40193010E94933669
:106A100079018A010894E108F1080109110985E06A
:106A2000FFEFEF16F1040105110591F188F162E124
:106A30007AE780E090E0A40193010E949336790107
:106A40008A010894E108F10801091109552011F0A3
:106A500086E001C084E02FEFE216F1040105110584
:106A6000B9F0B0F0C601B50120E034E040E050E0FC
:106A70000E94933679018A010894E108F10801091E
:106A80001109552011F087E008C085E003C081E0BE
:106A9000552019F485BD3AC082E08093B10036C01C
:106AA0005101CC24DD2460E072E18AE790E0A60188
:106AB00095010E94933679018A010894E108F10852
:106AC0000109110980E0E81680E0F80681E0080776
:106AD00080E0180710F491E010C068E478EE81E0DF
:106AE00090E0A60195010E94933679018A010894ED
:106AF000E108F1080109110993E0A1E05A1631F407
:106B000080918100887F982B9093810089819A8160
:106B1000AB81BC810097A105B10529F48FEF9FEFF0
:106B2000AFEFBFEF13C0220C331CB10180E090E047
:106B300029813A814B815C810E943F3628EE33E007
:106B400040E050E00E947136C901DA01E1E05E16D2
:106B5000A1F0F2E05F1619F1552099F5E7BC80939A
:106B6000C5059093C605A093C705B093C80580914D
:106B70006E00826080936E0024C0F0928900E092E3
:106B800088008093CC059093CD05A093CE05B0935B
:106B9000CF0580916F00826080936F0012C0E092F9
:106BA000B3008093D3059093D405A093D505B093FB
:106BB000D6058091700082608093700002C084E0EE
:106BC0006CCF0F900F900F900F90CF91DF911F918E
:106BD0000F91FF90EF90DF90CF90BF90AF909F907C
:106BE0008F907F906F905F903F902F900895EF92DD
:106BF000FF920F931F937B018C0161157105810535
:106C0000910529F420E030E040E050E00BC00E9404
:106C10000118A80197010E949336AC01CB01DA015B
:106C20009C01AD01B901CA011F910F91FF90EF9036
:106C30000895EF92FF920F931F937B018C016217CF
:106C400073078407950764F4261B370B480B590B11
:106C5000CA01B9010E94F735E60EF71E081F191F79
:106C6000B701C8011F910F91FF90EF900895009711
:106C700029F0BC0180E090E00E9406180895629F10
:106C8000D001739FF001829FE00DF11D649FE00D24
:106C9000F11D929FF00D839FF00D749FF00D659F85
:106CA000F00D9927729FB00DE11DF91F639FB00D84
:106CB000E11DF91FBD01CF011124089597FB092E95
:106CC00007260AD077FD04D049D006D000201AF458
:106CD000709561957F4F0895F6F7909581959F4F38
:106CE0000895A1E21A2EAA1BBB1BFD010DC0AA1F0D
:106CF000BB1FEE1FFF1FA217B307E407F50720F025
:106D0000A21BB30BE40BF50B661F771F881F991F9F
:106D10001A9469F760957095809590959B01AC01E8
:106D2000BD01CF01089597FB092E05260ED057FD12
:106D300004D0D7DF0AD0001C38F450954095309528
:106D400021953F4F4F4F5F4F0895F6F790958095EF
:106D5000709561957F4F8F4F9F4F0895AA1BBB1B66
:106D600051E107C0AA1FBB1FA617B70710F0A61B4B
:106D7000B70B881F991F5A95A9F780959095BC016C
:106D8000CD010895EE0FFF1F0590F491E02D0994B9
:106D90002F923F924F925F926F927F928F929F922B
:106DA000AF92BF92CF92DF92EF92FF920F931F9319
:106DB000CF93DF93CDB7DEB7CA1BDB0B0FB6F894CA
:106DC000DEBF0FBECDBF09942A88398848885F840A
:106DD0006E847D848C849B84AA84B984C884DF807B
:106DE000EE80FD800C811B81AA81B981CE0FD11D5F
:106DF0000FB6F894DEBF0FBECDBFED010895F89435
:106E0000FFCF2020202020202020202020202020F4
:106E100020200043572D506172746E657220005619
:106E2000312E3237005665722E203332382C2044F2
:106E30004C384B464F3B0053657475703A004765BC
:106E400073636877696E6469676B6569740057502E
:106E50004D202831302D3630293A0020200044754D
:106E60007263686761656E6765002832352D35305D
:106E700030293A00546F6E686F65686500546F6E14
:106E8000686F6568652028487A29003530302D31D3
:106E90003230303A004661726E73776F72746800F8
:106EA000446F74733A0041757367616E6700202008
:106EB000202020202065787465726E00202020201C
:106EC000202020696E7465726E00496E746572616F
:106ED0006B746976002020202020202061757300CB
:106EE0002020202020202065696E003565722D4706
:106EF00072757070656E00202020202020202020D8
:106F000020412D5A002020202020412D5A2C2030B5
:106F10002D390051534F2D4175737761686C0051C5
:106F2000534F2028302D00293A0048617570746D48
:106F3000656E75653A00576F7274747261696E6937
:106F40006E6700576F727465203A0051534F2D548D
:106F50007261696E696E670051534F204E722E3A0E
:106F600000576F7274652032205A65696368656ED8
:106F700000576F72746520322042533A00576F7287
:106F800074652033205A65696368656E00576F72B7
:106F9000746520332042533A00576F727465203471
:106FA000205A65696368656E00576F727465203496
:106FB0002042533A004C61656E6765726520576FD9
:106FC000727465005275667A65696368656E00352E
:106FD00065722D4772757070656E3A004B6F63680D
:106FE0002D4D6574686F64650028312D3339293A59
:106FF00020002020200020202020202020202020D1
:10700000202020202020202020200053657475702F
:1070100000010000000D003C008A02140032000153
:107020000001000100010033683B0000646B3B007D
:1070300000646C3B0000346F3B000035613B000096
:1070400036643B000039683B0000613B0000006390
:10705000623B0000636B3B0000636E3B00006374A7
:107060003B000064363B0000646A3B000065613B06
:10707000000065613B000065693B000065733B00F3
:1070800000663B00000066793B0000673B000000A3
:10709000676E3B000068323B000068613B0000689F
:1070A000623B000068763B0000693B0000006A34E8
:1070B0003B00006B3B0000006D3B0000006E3B009E
:1070C00000006F6B3B00006F6E3B00006F7A3B006F
:1070D0000070613B000070643B000073353B0000B2
:1070E00073763B000074393B000074613B0000750F
:1070F000613B0000756E3B000075723B00007672CC
:107100003B0000773B00000078613B000078763B55
:107110000000796F3B00007A333B00007A6C3B0043
:10712000007A703B00007A723B00007A763B0000E8
:1071300074663B000076753B00007673363B006A50
:10714000613B000078653B00007A733B00006C6196
:107150003B00006B3B006D3B00753B00723B0065E4
:107160003B00733B006E3B00613B00703B00743B97
:10717000006C3B00773B00693B002E3B006A3B0004
:107180007A3B00663B006F3B00793B002C3B00766E
:107190003B00673B00353B002F3B00713B00393B18
:1071A00000323B00683B00333B00383B00623B0051
:1071B0003F3B00343B00373B00633B00313B006406
:1071C0003B00363B00303B00783B003D3B0001FF7D
:1071D00000000000CE2D2B3243320000400014008E
:1071E000540000000000D7312B3243327C31A731EC
:1071F0008D31CB31FFFFFFFFFFFFFFFFFFFFFFFFE1
:10720000FFFFFFFFFFFFFFFFFFFFFFFFFFFFFFFF8E
:10721000FFFFFFFFFFFFFFFFFFFFFFFFFFFFFFFF7E
:10722000FFFFFFFFFFFFFFFFFFFFFFFFFFFFFFFF6E
:10723000FFFFFFFFFFFFFFFFFFFFFFFFFFFFFFFF5E
:107800000C94343C0C94513C0C94513C0C94513CE1
:107810000C94513C0C94513C0C94513C0C94513CB4
:107820000C94513C0C94513C0C94513C0C94513CA4
:107830000C94513C0C94513C0C94513C0C94513C94
:107840000C94513C0C94513C0C94513C0C94513C84
:107850000C94513C0C94513C0C94513C0C94513C74
:107860000C94513C0C94513C11241FBECFEFD8E036
:10787000DEBFCDBF11E0A0E0B1E0ECE9FFE702C060
:1078800005900D92A230B107D9F712E0A2E0B1E065
:1078900001C01D92AD30B107E1F70E942D3D0C945F
:1078A000CC3F0C94003C982F959595959595959582
:1078B000905D8F708A307CF0282F295A8091C0000B
:1078C00085FFFCCF9093C6008091C00085FFFCCF60
:1078D0002093C6000895282F205DF0CF982F809127
:1078E000C00085FFFCCF9093C6000895EF92FF92F1
:1078F0000F931F93EE24FF2487018091C00087FD22
:1079000017C00894E11CF11C011D111D81E4E8164B
:1079100082E4F8068FE0080780E0180770F3E09132
:107920000401F091050109958091C00087FFE9CF1E
:107930008091C6001F910F91FF90EF9008950E94D3
:10794000763C982F8091C00085FFFCCF9093C600B5
:1079500091362CF490330CF09053892F089597555D
:10796000892F08951F930E949F3C182F0E949F3CCF
:107970001295107F810F1F9108951F93182F882350
:1079800021F00E94763C1150E1F71F9108951F935A
:10799000182F0E94763C803249F0809103018F5F5E
:1079A000809303018530C1F01F9108958091C0003C
:1079B00085FFFCCF84E18093C6008091C00085FFE5
:1079C000FCCF1093C6008091C00085FFFCCF80E102
:1079D0008093C6001F910895E0910401F091050184
:1079E00009951F9108950E94763C803241F0809164
:1079F00003018F5F80930301853081F008958091AA
:107A0000C00085FFFCCF84E18093C6008091C00058
:107A100085FFFCCF80E18093C6000895E0910401CA
:107A2000F09105010995089540E951E08823A1F0FE
:107A30002D9A28EE33E0FA013197F1F721503040CA
:107A4000D1F72D9828EE33E0FA013197F1F7215064
:107A50003040D1F7815061F708953F924F925F9285
:107A60006F927F928F929F92AF92BF92CF92DF924E
:107A7000EF92FF920F931F93CF93DF93000080E16B
:107A80008093C4001092C50088E18093C10086E015
:107A90008093C2005098589A259A81E00E94143D24
:107AA00024E1F22E9EE1E92E85E9D82E0FE0C02ECA
:107AB00010E1B12EAA24A394B1E49B2EA6E58A2E50
:107AC000F2E57F2EE0E26E2E79E4572E63E5462E36
:107AD00050E5352E0E94763C8033B1F18133B9F107
:107AE000803409F46FC0813409F476C0823409F41B
:107AF00085C0853409F488C0803531F1823521F1A3
:107B0000813511F1853509F485C0863509F48DC0BC
:107B1000843609F496C0843709F403C1853709F423
:107B200072C1863709F466C0809103018F5F80932C
:107B30000301853079F6E0910401F0910501099582
:107B40000E94763C803351F60E94F33CC3CF0E94E2
:107B5000763C803249F78091C00085FFFCCFF092DF
:107B6000C6008091C00085FFFCCF9092C600809136
:107B7000C00085FFFCCF8092C6008091C00085FFC9
:107B8000FCCF7092C6008091C00085FFFCCF609250
:107B9000C6008091C00085FFFCCF5092C600809146
:107BA000C00085FFFCCF4092C6008091C00085FFD9
:107BB000FCCF3092C6008091C00085FFFCCFB09210
:107BC000C60088CF0E94763C863808F4BDCF0E945C
:107BD000763C0E94F33C7ECF0E94763C803809F4CC
:107BE0009CC0813809F40BC1823809F43CC1883942
:107BF00009F48FC080E00E94C73C6CCF84E10E94F2
:107C0000BD3C0E94F33C66CF85E00E94BD3C0E94D3
:107C1000F33C60CF0E94763C809306010E94763C44
:107C2000809307010E94F33C55CF0E94763C80333D
:107C300009F41DC183E00E94BD3C80E00E94C73C66
:107C400049CF0E94763C809309020E94763C809343
:107C5000080280910C028E7F80930C020E94763C79
:107C6000853409F415C18091080290910902892B8D
:107C700089F000E010E00E94763CF801E85FFE4FDA
:107C800080830F5F1F4F80910802909109020817AF
:107C9000190788F30E94763C803209F045CF809125
:107CA0000C0280FF01C16091060170910701660F0F
:107CB000771F7093070160930601A0910802B091AD
:107CC00009021097C9F0E8E0F1E09B01AD014E0F09
:107CD0005F1FF999FECF32BD21BD819180BDFA9A17
:107CE000F99A2F5F3F4FE417F50799F76A0F7B1F4B
:107CF00070930701609306018091C00085FFFCCF5F
:107D0000F092C6008091C00085FFFCCFB092C60003
:107D1000E1CE83E00E94C73CDDCE82E00E94C73CFA
:107D2000D9CE0E94763C809309020E94763C8093D3
:107D300008028091060190910701880F991F909386
:107D40000701809306010E94763C853409F4A6C0A1
:107D500080910C028E7F80930C020E94763C8032D0
:107D600009F0B8CE8091C00085FFFCCFF092C6002C
:107D7000609108027091090261157105B9F140E046
:107D800050E080910C02A82FA170B82FB27011C0E2
:107D9000BB2309F45CC0E0910601F0910701319624
:107DA000F0930701E09306014F5F5F4F46175707B7
:107DB000E8F4AA2369F3F999FECF209106013091E6
:107DC000070132BD21BDF89A90B58091C00085FFB2
:107DD000FCCF9093C6002F5F3F4F30930701209355
:107DE00006014F5F5F4F4617570718F38091C00099
:107DF00085FDE5CE8091C00085FFF8CFE0CE81E023
:107E00000E94C73C67CE0E94763C803209F08CCE3F
:107E10008091C00085FFFCCFF092C6008091C00029
:107E200085FFFCCFE092C6008091C00085FFFCCFAB
:107E3000D092C6008091C00085FFFCCFC092C600E2
:107E40008091C00085FFFCCFB092C60043CEE09188
:107E50000601F091070194918091C00085FFFCCF4D
:107E60009093C6009CCF80E10E94C73C33CE0E9415
:107E7000763C0E94763C182F0E94763C112309F430
:107E800083C0113009F484C08FE00E94C73C22CE29
:107E900080910C02816080930C02E5CE80910C02EF
:107EA000816080930C0259CF809107018823880F4D
:107EB000880B8A2180930B02809106019091070123
:107EC000880F991F90930701809306018091080203
:107ED00080FF09C080910802909109020196909359
:107EE000090280930802F894F999FECF1127E091D6
:107EF0000601F0910701C8E0D1E08091080290915D
:107F00000902103091F40091570001700130D9F34B
:107F100003E000935700E89500915700017001308D
:107F2000D9F301E100935700E89509901990009169
:107F3000570001700130D9F301E000935700E89534
:107F40001395103498F011270091570001700130FB
:107F5000D9F305E000935700E895009157000170B0
:107F60000130D9F301E100935700E895329602976A
:107F700009F0C7CF103011F00296E5CF112480919F
:107F8000C00085FFB9CEBCCE8EE10E94C73CA2CD19
:0E7F900085E90E94C73C9ECDF894FFCF80008B
:00000001FF
